:020000041100E9
:103000007FB50023284C294D03932800217C284AB2
:1030100001F0D9FA002812D103232800217C03AA49
:1030200001F078FA00280AD1224B039A9A4206D17D
:10303000214B2248E360224B636104B070BD02263D
:10304000217CFE2228001F4B009601F035FA002853
:1030500001D00020F1E71C4BA2899A42F9D1217CD2
:10306000FF222800194B009601F026FA0028F0D123
:10307000E389174A934203D1164B17486361DCE793
:10308000164A9342E5D1164B164A1B68934206D95D
:10309000C02304222800217C9B0001F076FA124B09
:1030A00012486361C9E7C046F461FF1F3442FF1F45
:1030B000813700005959530059598320B0BA001183
:1030C000F94100110062FF1F595900000262FF1F01
:1030D00083050000AD41001190BA00118215000077
:1030E0001862FF1F87130000B5420011A0BA00113B
:1030F000002370B51A4E1B4C30006361637401F0FD
:1031000089F9402323744B2B0CD9CC233821AC22D2
:1031100030009B01217401F038FA00280AD0002504
:1031200025740CE0FFF76CFF051E08D1237C0433E7
:10313000DBB2E7E70C4B0D4D63610D4BE381236878
:10314000002B08D1002D06D00C222900200008F009
:10315000EBFB2B7B6374300001F09AF970BDC04625
:103160003442FF1FF461FF1F4D42001180BA00116D
:10317000AAAAFFFFF7B5164B0192C318021D002043
:10318000009388235B05D3181B685C1C1AD09CB283
:10319000402C18D88D781E0CAC466746CD782D0291
:1031A0003D43AE4206D1019800280ED110000C70AC
:1031B000240A4C7003249BB20733A343D218009B0C
:1031C0009A42DED3FEBD4432F9E71000FAE7C0466A
:1031D000FC0F0000802213B503000324019189B283
:1031E000520107319B18A14304305A1A88235B050A
:1031F000C3181B68591C03D190429241104016BD60
:1032000099B2402907D80B000733A343C018904256
:10321000ECD30020F3E74430F9E7134B134A1B6863
:10322000126810B5FA24934201D81A00F824104B02
:10323000E4021B689A4210D813000E4A12689A42A0
:103240000ED3013307D1F823DB029C4203D10A4994
:10325000054808F099FB200010BDFC24E402ECE7CF
:10326000FE24E402F7E7C04600C0071100D00711B2
:1032700000E0071100F00711FFFFFF7FF0B59BB0E2
:10328000150004900391402A00D9A0E006AB5980B4
:103290001A80FFF7C2FF0400042816D9002206A9ED
:1032A000FFF768FF052810D906AB1B88AB420CD18D
:1032B000002D07D0514B2A000499C01808F0C4F81B
:1032C000002802D101201BB0F0BD06AB1D802000FC
:1032D0000699FFF77FFF041E7BD1069B0793FFF73C
:1032E0009CFF80235B01C618802307001B039E42BE
:1032F00001D3F826F60288235B05F31801931B68B7
:10330000013302D0019808F037FA3D49019808F0DE
:103310003BFB3B1D0293331D05938822029B520504
:103320009B181B6808935A1C3CD044219AB2009108
:10333000402A04D80320D11D814389B2009103990A
:103340001B0C8B4224D0402A22D80122300008A92D
:10335000FFF710FF021E1BD1380008A9FFF70AFF74
:103360000400042831D9009A059B9B188022520141
:10337000B218934240D288235B05C118009A09A86D
:1033800008F0D2FA1D4B009A09A9F01808F00CF8C1
:10339000009A029B9446634402931A4B029AFB18CC
:1033A0009A42BAD388235B05FC1821680198013939
:1033B00008F0EAFA200008F0DFF9039A07AB5A8018
:1033C00030000799FFF706FF0400002C03D100200E
:1033D00079E70428FBD988235B05E018069908F0F3
:1033E000D3FA0323EA1C9A4300D16BE7034B0499F9
:1033F000E01807F0D9FF65E70424ECE704000011AA
:10340000FFFFFF7FF80F0000F7B505001400402A0A
:1034100021D8002701AE71803780FFF7FEFE042817
:1034200016D93A003100FFF7A5FE042810D93688D6
:10343000BC420BD0BD4209D0221CB44200D9321C80
:10344000064B92B2C118280008F06EFA30B2FEBDE9
:10345000C04300B2FBE703204042F8E7040000113C
:1034600037B5042204000D0001A81649FFF7CCFF70
:10347000020004280BD1019BA34208D3AB4204D025
:10348000104901A80195FFF7F9FE01203EBD0E4C41
:1034900023682000019308F06FF901992000013999
:1034A000019108F071FA80235B01E418074B9C42FC
:1034B000EED10422034901A80195FFF7DFFE0020A9
:1034C000E4E7C0465555000000C007110000081190
:1034D00030B589B008F018F810226946254808F080
:1034E00053F9254B009A9A420ED1019B029A0F2B59
:1034F00033D8002101240698013B08D2002900D0CE
:103500000292029B013331D10023029325E0551C26
:10351000F2D102002100EFE710341022200004A9AC
:1035200008F032F9029B013301D1069B02938823F4
:1035300004995B05C918059B06981A03120B0491A0
:103540000592814203D02B4201D108F0EDF9019B95
:10355000013B0193019B002BDED1029B002B03D08A
:10356000049304984168084709B030BDE025014C38
:103570002D03EFE700000111504859368022F8B5BD
:10358000964C974BD200002120001C6007F0E4FE0F
:103590002300944A88331A60934B1A786A23002ACE
:1035A00000D01133E3620A232365904B37221B7846
:1035B0000820A3638E4B2118E361102323628D4BF7
:1035C0003B256361C823DB00A36123008C331A60B1
:1035D0002823013AE26320646364CA67043A211D28
:1035E000CA672100BC310D602100C0310860210094
:1035F000C4310B6021000635CC310D602100083D3F
:10360000C8310D602100D0310A602200D432106030
:103610002200D832136022000227E0322100176016
:103620004222DC310A6021001B3DE4310D602100A3
:10363000E83108602100EC310B6023000521F433F0
:1036400019602300F0331A602300183290331A6097
:1036500023009433186023001E3A98331A60AF2376
:10366000DB002360644BFA262363644B644DE36004
:10367000644BF031A3642300FF31FC33B600A1603A
:1036800021611E60A5627325E5656D3D6565A565D3
:1036900096255D4AAD00E264666258606766A5667D
:1036A00000270925A767E566584F594D6067200038
:1036B0002567E2673A6015279C30676007001A208B
:1036C00038602000A0300700212038602000A8309A
:1036D00007004C4838602000F83006602600642758
:1036E000A436376026005F3FAC3637602600033FC4
:1036F000B03637602600C637B4363760260000275C
:10370000B836376038269E60424E96205E64424E40
:103710005A66DE61414E9A645E62F53EFF3E9E62ED
:103720001E269A67354A8000DE661F675F67DD6583
:103730001D661862DA67BE23394A5B00E250394BD6
:10374000D838235004302250C4225200A350C6233C
:10375000E4205B00E1500433334AE1503349344BF9
:10376000D1603449800019503349E938FF38195085
:1037700032490430195032493248D161324911631B
:10378000324951631900F4310860CE2030494000BD
:1037900011603049195019002F48F83108602F493D
:1037A000D16582212E4A89005A501A002D490832CB
:1037B000D1671A002C49B432116088212B4A890044
:1037C0005A501A002A49883211602A4ADA6408F0ED
:1037D000C3F8012007F008FEF8BDC0460004FF1F33
:1037E0009064FF1F606FFF1F6444FF1F4A0AFF1FA2
:1037F0003A07000080C3C9019A020000DC050000FE
:103800006A18000050C3000088130000F009FF1F71
:10381000204E00006509FF1F68100000C409000069
:1038200040420F0010270000FC00FF1FB11CFF1FCB
:103830000000FF1F052DFF1F8D30FF1F252FFF1FCD
:103840007120FF1F6127FF1F8D20FF1F3922FF1FDF
:10385000FD1FFF1F8529FF1F6D2AFF1F8D19FF1FE9
:103860009128FF1FB525FF1FC125FF1FFD1EFF1F4C
:10387000B51FFF1F751EFF1F0223F0B50124624D07
:10388000624E2B70624B91B01C70624F0393336891
:10389000002104207B7006F05BFC042006F052FB44
:1038A0000023984205D07A78552A02D0332A00D0D6
:1038B0009DE03360042006F0C5FD07F0DDFDFFF755
:1038C0005DFE08F011F81F2201240021524B10AEBA
:1038D0001A70524B1C70524B1970524B196891431D
:1038E000163A0A431A60602219689143403A0A4323
:1038F0001A6007F0B9FF07F017FE4B4B9847C1203D
:10390000FF214A4B80001A588A431A50C522920060
:1039100098588843BF390143995098584449084002
:103920008021C9010143802099509958C00509029E
:10393000090A0143995080213E48490107F0CCFE15
:10394000032322003C49019400933C4807F0C4FD46
:103950002C223B4905A807F0E7FF05AC61782078E9
:10396000023406F00FFBA642F8D1364C112000219C
:1039700006F01CFC2268344B03201A40A023DB0213
:1039800013432360802322689B041343236022682F
:103990002E4B1A4080239B03134323602C4A2D4B4C
:1039A000934200D8012007F05FFD07F095FF8023C8
:1039B0002268DB0413432360287807F0D5FF039BBC
:1039C0001878C0B207F050FE07F01EFD224904200F
:1039D00007F0DAFD06F002FD00F040F800F00CFE02
:1039E00000F0B4FE00F010FA002011B0F0BD00931A
:1039F0002100194A042007F057FE8023DB059C6252
:103A0000FFF766FD56E7C0464A0AFF1F34F0004044
:103A10006444FF1F2462FF1F480AFF1F490AFF1F5B
:103A2000680AFF1FBCF00040E1A2000000E100E0D6
:103A3000FF00FFFF6844FF1FEC56FF1F6854FF1F85
:103A4000A8B9001114F00040FF7FF8FFFFFF9FFFAF
:103A50000080FF1F606FFF1F3B000108002210B5B0
:103A60001100112007F098FC10BD0000002370B574
:103A70000925334E334C3362E3681120AB43E360D6
:103A800007F082FC112007F057FF112007F0CCFD52
:103A90004023226811201343236080236268DB02E5
:103AA000134363608023A2681343A360A368264A7C
:103AB0001340A3608023A2689B0113431022A360DC
:103AC000236C934323640123226C1A4322648022D3
:103AD00052003262216B1D4A11402163616B11401B
:103AE0006163A16B1140A163E16B0A40E263E2688C
:103AF00017490A40E260174A11680B43136007F048
:103B000013FEFD21144B154A89005A508023C7200B
:103B1000626B5B0313436363E36880001D43104BD8
:103B2000E56019580F4A1140802212020A431A50C8
:103B3000802292051A6008220B4B5A6370BDC04662
:103B400000F000403CF00040FFFFDFFFEFFFEFFF21
:103B5000FFFF7FFF003800400000FF1F5118FF1FCC
:103B600000E100E0FF00FFFF00000540E12010B58C
:103B7000C00407F0C1FD10BD70B52B4C238C002B89
:103B80002AD0FA22D200934201D2FFF7EFFF228A15
:103B9000238C002A21D1DA0023826382A382E3826C
:103BA00023836383A383E38322606260A260E26075
:103BB0001E4D1F4A6420EB8093420AD8FA2200204F
:103BC000D200934205D91B4A0A21981807F004FD38
:103BD000C0B200232872238470BD0720E11CCA7F75
:103BE00001320240CA7705D10325201DC17F013172
:103BF0002940C17708325200A352002321001A0045
:103C0000088A01321B180231082AF9D1221DD27FFD
:103C10009200A350626823689B18A2689B18E26810
:103C20009B185B099BB2C3E76461FF1F0C62FF1F17
:103C3000B70B000030F8FFFF30B503A804880B2055
:103C4000002C0ED14968074D0878497809020143D4
:103C50000A20A94205D1012120001980024B1B7ABC
:103C6000137030BD192A00000C62FF1FF7B5150054
:103C700008AA16884A680F4F147852781202224315
:103C80000A24BA4214D10122DBB2019200962A0022
:103C900007F0F4FA041E0BD1074B1B68002B07D06A
:103CA00068782A7800021043424250410130984718
:103CB0002000FEBD022900009061FF1F30B50125E4
:103CC00003790400BFB02B4211D00A49408806F0A6
:103CD00041FE28420BD0084B01A95B8D4D800B8023
:103CE000064B00221B7A60880B7103F013FF3FB074
:103CF00030BDC0468861FF1FA840FF1F0C62FF1F38
:103D000010B50549054806F0DBFD0421044A0548C5
:103D100006F098FD10BDC0468861FF1FFFFF000040
:103D2000D4B90011A840FF1F10B5024804F074FD7B
:103D300010BDC046BD3C0011012303700B4B1A7A25
:103D40004270022282709A78C270DA78027103227D
:103D500042711A7982715A79C2710C2202729A796F
:103D60004272DB7983720B207047C0460C62FF1FE2
:103D7000022310B50370013B437005338370103389
:103D80000371443B43712A3383714433C37100236D
:103D90000372064B04001B8843720A30FFF7CCFF06
:103DA000831D0A30C0B2E37010BDC0460C62FF1F15
:103DB00010B5142007F040FC124B142200211860AB
:103DC00007F0CAFA002007F0A7FD012007F0C4FBA6
:103DD000022007F0D1FB032003F0C2FF042005F00E
:103DE000D7FF052003F000FA062003F0CDFE0720E0
:103DF00001F064FA082006F005FD092001F040F802
:103E000010BDC0469461FF1F07F0B6FD012007F00A
:103E100083FC07F091FB0000094B10B504009842A9
:103E200005D0012904D12000064906F049FD10BD46
:103E30000229FCD1013904F0ADFC0028F3D0F6E7EB
:103E4000FEFF0000BA61FF1F70B50D7A100004AAD2
:103E50002C00168810221440154220D1002E20D1AB
:103E60000A78022A18D14A68517815780E4A090250
:103E70002943914205D00D4A914209D01C800A2461
:103E800004E014220A491A8007F04EFD200070BD9C
:103E90000C2208491A80F7E71C800124F6E7082461
:103EA000F4E70B24F2E7C046F3FF0000F4FF000044
:103EB000F042FF1FCCBA001110B5040007490848B2
:103EC00006F0FEFC074804F0E7FB0020E40704D5F9
:103ED0000721054A054806F0B5FC10BDBA61FF1F71
:103EE000FFFF0000193E001118BA0011EC40FF1F3F
:103EF00000B50C4BBFB01A780B4902A800F0E0FCEB
:103F00006B4680B2D880002809D06A46074B01A9C9
:103F10001B889380064B0022188803F0FBFD3FB0FE
:103F200000BDC0469861FF1F9961FF1F4641FF1FFA
:103F30005042FF1F00B50C4BBFB01A780B4902A8C6
:103F400001F02EFD6B4680B2D880002809D06A4669
:103F5000074B01A95B8D9380064B0022188803F064
:103F6000D9FD3FB000BDC046C261FF1FC361FF1F46
:103F7000EC40FF1F5042FF1FF7B50E00377A1C00C0
:103F800008AB11003D001A8820231D401F423CD180
:103F90003378022B3BD173681F785B781B023B435D
:103FA0001E4FBB4208D01E4FBB4214D01D4DAB422A
:103FB00021D00A252800FEBD002A2AD1142C2AD897
:103FC0002200F06807F0B0FC174B1C70012CF1D9EF
:103FD000FFF7B0FFEEE7002A1BD1202C1BD82200F0
:103FE000F06807F0A1FC114B04211C70104B1878ED
:103FF00007F032FADEE7E3B20124009201940A00EE
:10400000310007F03BF90500D4E70825D2E7012588
:10401000D0E70B25CEE70D25CCE7C046F3FF000027
:10402000F4FF000002290000C261FF1F9861FF1F1A
:104030004462FF1F332310B5040003700A220749AE
:10404000013007F071FC064B0F201B681A0AE3725F
:1040500022731A0C1B0E6273A37310BD0C62FF1F38
:104060003462FF1F30B5012503790400BFB02B4235
:1040700013D00B49408806F06DFC28420DD06A46EB
:10408000084B02A81B889380FFF7D4FF6B46D880AB
:104090000022608801A903F03DFD3FB030BDC0465D
:1040A000BA61FF1F4641FF1F10B5024804F0B4FB80
:1040B00010BDC0466540001170B5160004AA1488F2
:1040C00005AA15784A685078117800022A4A0843F0
:1040D000801805284BD807F06FFB03131E29343FC7
:1040E0000720032C0BD80422121BAA4200D92A0055
:1040F00022491A803000091907F016FC002070BD13
:104100000720112CFBD81222121BAA4200D92A0028
:104110001B491A80EEE707200E2CF0D80F22121B45
:10412000AA4200D92A0017491A80E3E70720032C86
:10413000E5D80422121BAA4200D92A0012491A808B
:10414000D8E70720032CDAD80422121BAA4200D990
:104150002A000E491A80CDE70720032CCFD804226D
:10416000121BAA4200D92A0009491A80C2E700227C
:104170000A201A80C3E7C046DCD5FFFF63BA0011EE
:10418000E061FF1F53BA00114EBA001149BA001185
:1041900044BA001110B50D21024A034806F052FB43
:1041A00010BDC04638BA00115C41FF1F13B5104C5A
:1041B0000423217C01AA00F0ADF9002815D16B463B
:1041C0009A88236852BA92B25343228909491B0C38
:1041D0009B184B806B46DA88636852BA92B253439D
:1041E00062891B0C9B188B8016BD0120FCE7C04622
:1041F000F461FF1F0C62FF1F13B5124C06236A46C1
:10420000217C00F087F9002819D16B4619882368B2
:1042100049BA89B24B4321890B4A1B0C5B18538066
:104220006B46D97803335B781B020B435BBA61683A
:104230009BB24B4361891B0C5B18938016BD012018
:10424000FCE7C046F461FF1F0C62FF1F37B5174C37
:1042500007236A46217C00F05DF9002824D16B46D3
:104260001B787F2B20D86B46DD78F0232A041B03B4
:104270001A406B469B880E495BBA9BB21A4323686F
:104280002D09534322891B0C9B184B806B465A788F
:104290009B7812031B011A4363682A4353436289C4
:1042A0001B0C9B188B803EBD0120FCE7F461FF1FB7
:1042B0000C62FF1F7FB50226154C0022217C03AB48
:1042C0000096050000F0F8F8002802D0012004B0A4
:1042D00070BD0E23217C0122280000966B4400F063
:1042E000EBF80028F2D16B469A892368D2BA53437F
:1042F000228908491B149B184B806B46DA89636836
:1043000052BA92B2534362891B0C9B188B80DEE732
:10431000F461FF1F0C62FF1F70B5184C237C002B4B
:104320000FD0382B0ED1164D280000F073F8CC2397
:10433000AC222800217C9B0100F027F9280000F026
:10434000A7F870BDE3890F4A934209D10C4D2800AC
:1043500000F060F800222800217C00F005F9EDE76C
:10436000094A9342EDD1064D280000F053F89022FF
:104370002800217C920100F026F9DFE7F461FF1F9D
:104380003442FF1F830500008320000070B5144CE9
:10439000237C002B1FD06369002B1CD0114D2800FB
:1043A00000F038F86369280098470400280000F0FE
:1043B0006FF8002C10D10C4B0422995E002905DA0D
:1043C0009C801A8801321A80200070BD074A9142F1
:1043D000F7DD9A80F5E70124FEF78AFEF4E7C04690
:1043E000F461FF1F3442FF1F0C62FF1F0F27000004
:1043F00010B58024064AA4001168436B234205D1FE
:1044000013685B1A032BF8D9012010BD0020FCE7CC
:104410006008FF1F70B5C17905000C00631E9C4148
:104420001A4BE402E41849000460C9B2007905F0AF
:10443000F3FEE979687949000131C9B205F0ECFE73
:10444000E8790930C0B207F0EFF80023E366613382
:104450002360AA795B3B002A0ED022689A43023B74
:10446000134323600A23E36107332362002323639A
:10447000A3630133E36370BD22689A4302231343AD
:104480002360462363610633A361EFE700500040D9
:1044900070B5002504000368DD66C0790930C0B23C
:1044A00006F072FF2900207905F052FE290060799C
:1044B00005F04EFE70BD0000F8B51E0006AB1D787D
:1044C000002304681700E366616007F01DF801230C
:1044D0008022E3662B0027615200013B08D207F0DF
:1044E00093F908200A4A1168002D03D12800F8BD6D
:1044F0002261F2E7236F034203D02369013D337049
:10450000013613685B1A032BEED90125EEE7C0468E
:104510006008FF1F70B51C00002305681600EB66DD
:10452000696006F0F1FF01238022EB662300520050
:10453000013B08D207F068F908200A4A1168002CEC
:1045400003D1200070BD2A61F2E72B6F034203D034
:104550002B69013C3370013613685B1A032BEED9CB
:104560000124EEE76008FF1F002370B50468150002
:10457000E366616006F0C8FF0123E366256107F08A
:1045800043F92000FFF734FF70BD70B51D00002314
:1045900004681600E366616006F0B6FF0123E36677
:1045A00026610F33626B1A42FCD02B0A2361102361
:1045B000626B1A42FCD0EDB2256107F025F92000AC
:1045C000FFF716FF70BD002370B504681500E366A1
:1045D000616006F099FF0123E3662B0A2361102333
:1045E000626B1A42FCD0EDB2256107F00DF9200094
:1045F000FFF7FEFE70BD000010B5084CE368002B0D
:1046000008D18022064B52021B689B186360054B41
:104610001B68236007F020F9A06010BD3462FF1F03
:10462000C8F00040CCF0004070B5184A936A916A17
:104630009942FBD116498A689A421FD39A1A8B6015
:10464000144B0126186893B2D202D20E4343424360
:1046500000204C681B0A1B1912029B180E4C0A689A
:104660004B60551CA3420CD8002801D04B600A6057
:104670000A4A136008680A4B186070BD581E821AF7
:10468000DDE7084A30009B182A00EAE700F0004006
:104690003462FF1F140AFF1F40420F00C8F00040A1
:1046A000CCF00040C0BDF0FF70B51F4C23793F2B0C
:1046B00001D93F2323711D4B22791A701878C0B29B
:1046C00006F012FF18231A491A4A0B801A49138060
:1046D0000B805380A379194980200B800C21938093
:1046E00001334B43164D191C0001834200D9011CB4
:1046F0002980D1806379002B01D101336371237A42
:10470000012B01D8022323726279237A0D48534387
:104710000A21584306F060FF0B4D2860E379052B12
:1047200001D81023E37170BD2862FF1F480AFF1FE4
:104730004E42FF1F1044FF1F4C42FF1F4A42FF1F03
:104740004842FF1F710200001862FF1FF8B52021C8
:104750000020FEF785FE114C011E114D09D10C22DF
:10476000104BC1CBC1C4280006F0F6FDFFF79CFF3B
:10477000F8BD0C2220000C49FEF746FE0C2802D0A2
:10478000084B43CB43C40C2228000849FEF73CFEEB
:104790000C28EBD00C220021E5E7C0462862FF1F61
:1047A000F461FF1FC0BA0011FC0C0000F50C000002
:1047B000F0B51D4C8022A5440400882069465201B2
:1047C000400506F019FF902212016A4413002000F0
:1047D00032C832C316C816C38023144C144FA668BF
:1047E0009B033343A3603B6006F0BEFE8823A068B2
:1047F0005B05C01806F0C0FF002588232900802231
:10480000A0685B05C01840196944520006F0CCFD51
:1048100080230135FF355B019D42EED1A6603E60ED
:10482000044B9D44F0BDC046FCEFFFFF8043FF1FDB
:104830009808FF1F04100000F0B5040087B000289E
:1048400025D0684606F0B8FD1B4C022806D106228A
:104850006946200006F0F8FD002816D069460023BE
:1048600001250F262F00E25C01331009103087402C
:1048700038002F00324097403A0002434A61043921
:10488000062BEFD16846FFF793FF07B0F0BD182263
:1048900069460A4806F0B0FE6A46A300D3580133C1
:1048A00005D01822FF21684606F056FDEAE70134DC
:1048B000062CF1D1E9E7C0466509FF1F0009001188
:1048C000F0B5002504000E0085B0AA4200D183E0B7
:1048D0004B1C087801934B78897837790902194382
:1048E000F3783F061B040B431F430397207065704A
:1048F000252800D193E033D8112813D806F034FDD1
:1049000066001701170117011701A700B500AE00D7
:1049100017011701170117011701170117011701D7
:10492000F1001101232800D1CAE0DB2800D020E1EA
:10493000042A00D8AEE01025052A05D0551F2A000C
:104940003800711D06F0F0FF05223100200006F04E
:10495000EBFF2A003900601D06F0E6FF05353BE05D
:10496000562856D010D8332800D1A4E0552836D088
:104970002628DAD18E4B2900132218001D0006F0DC
:10498000EBFCFEF7B5FB59E0712800D174E072280A
:1049900000D186E0DC28C8D1022A00D87AE07378FA
:1049A000BFB26370B378A370032A05D0033A39000D
:1049B00092B2F01CFEF762FC10223900E01CFEF7F8
:1049C00023FDC51C002807DA607070E00C2220006F
:1049D000784906F0A9FF0C25280005B0F0BD013A82
:1049E000754D0C2A13D8002A0AD02800019906F028
:1049F0009BFFFFF759FE0C2228007049FEF73EFC92
:104A000029000C22601C06F08FFF0D25E4E70C2224
:104A1000EBE7694D6A4B2A0043CB43C2E9E7013A11
:104A2000634D0C2A11D8002A08D00199280006F0FD
:104A30007BFF0C2228006349FEF720FC290013228B
:104A4000601C06F071FF1425C6E70C22EDE7062274
:104A50005D49601C06F068FF0625BDE712225B4930
:104A6000601C06F061FF1325B6E708225849601C58
:104A700006F05AFF0925AFE7012A0ED07178F02918
:104A800008D8544D288801F0E7FB534B2A88520080
:104A9000D35A00E0FF23637009E04E4A4E4B128860
:104AA000F5E74E4B012A04D072781A706270022525
:104AB00092E71B78EFE72000FFF7BCFA05008BE7D1
:104AC000042A04D9464D2F6006F0C6FEA860FFF701
:104AD000ABFD0422039003A9601C06F025FF052509
:104AE0007AE7404D062A15D906222800019906F0DA
:104AF000ABFC00280ED006220199280006F014FF16
:104B0000062239492800FEF7B9FB0123334A117800
:104B10000B43137029000622601C06F005FF0725D1
:104B20005AE7012AB6D07078FFF786FEBFE7012862
:104B300000D0FAE6931E2D4F132B06D87378002B66
:104B40000BD100F00BF900F041F9294B39001D7829
:104B5000601C6A1E06F0E8FE3EE7551E2A00019919
:104B6000380006F0E1FE38002249AAB2FEF786FBC3
:104B7000E9E7DA288ED1042A8CD9082A15D9B37925
:104B800072791B021343F27912041A43337A1B061B
:104B900013433B603B68052231002000039306F07D
:104BA000C3FE0422601D03A962E7FE236370F1E7E0
:104BB000F461FF1FCCBA00112862FF1FFC0C00003B
:104BC000C0BA0011F50C00000062FF1FE061FF1F7A
:104BD0008443FF1F5042FF1F9464FF1F2462FF1F86
:104BE0003462FF1F6509FF1FADAC00002564FF1F85
:104BF0002364FF1FAEDE000070470000020010B506
:104C0000094B0A32094C92B2DA815A829881188291
:104C1000207802F087F90422054B012120781A70D0
:104C200006F01AFC10BDC0460E43FF1F6E64FF1F46
:104C30006D64FF1F013870B5042809D806F0BCFD6B
:104C40000309230812001E4B0221187806F004FC09
:104C500070BD1B4B0821187806F0CEFB0022194BC3
:104C60001A72F5E780220024164B154D52001A8166
:104C7000082128781A68DC7206F0EEFC21002878FA
:104C800006F0A2FDE4E70E4B0821187806F0B4FB0D
:104C90000D48FFF76DF80D4B0D4A9B7993800D4A37
:104CA00013800022074BDA720132FF321A810A4B5D
:104CB0001B78002BCCD0094A136006F06DFDC7E7C6
:104CC0004462FF1F1862FF1F5942FF1F2862FF1F27
:104CD0001044FF1F4A42FF1F2462FF1F34F00040B0
:104CE00010B500290ED104280CD10D3005F05EFA64
:104CF000054B1B78002B05D02622044B04485A7222
:104D0000FFF77CFF10BDC0464664FF1F1862FF1FFF
:104D1000C409000010B5012904D1042802D10D30C6
:104D200005F044FA10BD00000300F0B50A4D8E18DE
:104D3000B14202D152008018F0BD0C782F682409CE
:104D40003C5D0F271C700C7801313C402F683C5DA6
:104D50005C700233ECE7C0464442FF1F0D22124B49
:104D600010B51A700C23114C11492370093A033BFA
:104D70001048637006F0D8FD2D2301220E490F481C
:104D8000A371FFF7D1FF01220D49FFF7CDFF0122EB
:104D90000C49FFF7C9FF030000200B4902001870FF
:104DA000FEF76CFA10BDC0464264FF1F2364FF1F6C
:104DB00063BA00112564FF1F6709FF1F2A64FF1FE4
:104DC0006609FF1F6509FF1FAEDE000070B5134CBA
:104DD000142220001249FEF717FB431E114D132B1E
:104DE00019D8AB78002B16D0431C2B7009236B709D
:104DF00000230019037028780B4B01302900C0B242
:104E0000187006F0D9FB297822000139C9B20020B8
:104E100005F036FC70BDFFF7A1FFECE72564FF1F2E
:104E2000AEDE00002364FF1F4264FF1F10B5114B6C
:104E30001A781870002A0ED000280BD10E4B1A7861
:104E4000062A07D85423D340DB0703D50B4B187829
:104E500002F068F810BD0028FCD0074B1B78012B2E
:104E600002D0033B022BF5D8044B0121187806F041
:104E7000F3FAEFE74664FF1F6D64FF1F6E64FF1FC8
:104E800070B54D4E4D4A4E493070042005F084FAFD
:104E90000021112005F08AF9112005F06BFAFEF7C8
:104EA00027F906F0C9FA032246494748FFF73CFFB5
:104EB0002D24030004221C7044490130FFF734FF05
:104EC00030230470424D434C437083702E3B0622C6
:104ED00020004149EB87FEF797FA062813D02000FF
:104EE00006F06AFA022809D00321200006F0D4FA5D
:104EF0008D23E3706E3B237119336371062220000A
:104F00003549FEF7BBF9354B1B68FC335C64FFF792
:104F10005DFF0020FFF78AFF314C324A0121324BFE
:104F20001278207801F0C0FF304A314B127800210E
:104F3000207801F0B9FF01222E4B1A702E4B5B78BE
:104F4000552B31D12D4B3B325A722D4B2D4AAB8113
:104F5000EA812B826A822021307806F0EDFB012065
:104F6000404205F0D9FB0120404205F075FCFFF7F7
:104F700011F9FEF7C5FE00F0ABFC01204042FEF740
:104F80009BFF012006F038FCF02001F049F90121D7
:104F9000307806F061FA307802F020F91A4806F00D
:104FA00023FCFEF763FD70BD6422184B5B7953430D
:104FB0001A000A32CBE7C0464462FF1FE14C0011E1
:104FC000154D00118443FF1FE061FF1F0062FF1FAA
:104FD0000E43FF1F6509FF1FADAC00009064FF1F6B
:104FE0006E64FF1F7842FF1F5942FF1F4264FF1F7C
:104FF0002364FF1F1464FF1F2462FF1F1862FF1F3A
:10500000C4090000CE0900004662FF1F2862FF1F8E
:10501000F8B50A0020230D001A4019425DD05A4B02
:105020001B78002B42D0FFF7FFFA584B584C594ED3
:1050300099686268737A8A1ADB039A4202D36160C4
:10504000FEF714FD327A217A531EDBB2994230D139
:10505000FFF762F9637A002B25D0013BDBB2637264
:10506000002B20D14C4B5B78552B01D106F094FBE3
:10507000E37A002B12D00023A27AE3729A4202D084
:10508000A372FEF779FD454A454F13883800013376
:105090001380FEF76DFE390006F02EFA6423707956
:1050A0005843FFF7ABFD237A013323722020684079
:1050B000F8BD9142CED300272772FFF767F9A37A94
:1050C000BB4202D0A772FEF757FD354F3800FEF7FE
:1050D0004FFE390006F010FABCE70BB2002B0ADADB
:1050E000304B187806F030FC002801D006F0E4F9C7
:1050F00080200002DBE70224214206D0244B01205D
:105100001A72FFF793FE2000D1E70B071BD5FFF7BC
:105110008BFA1E4B1E491F4C98684A68637A821AA4
:10512000DB039A4202D34860FEF7A0FCFFF72EF99A
:10513000FFF7F2F800F0E6FB2368DB0701D5FEF786
:10514000B3FF0820B3E7CB0609D5FEF715FD0E4BDC
:105150001B78002B01D1FEF7E7FD1020A7E7012403
:10516000214209D0104800F06DF806F01DFB210027
:10517000112005F01BF8C6E7042408002040214256
:1051800096D0FEF7B5FEBEE74664FF1F3462FF1FF0
:105190001862FF1F2862FF1F2462FF1F0C62FF1F9F
:1051A0005942FF1F4462FF1F3C42FF1FF0B51B4BDB
:1051B0001B4F1B883A8804001A4E1B4D85B09A423B
:1051C0000DD832889A420AD3184B1A882B889A42F3
:1051D00005D1174A174B12881B889A421BD005200D
:1051E00001F074F83B8802AA138033880190538041
:1051F0002B88114D93800F4B02A91B88D3800F4B36
:105200002A78188802F090FD0D4B08212878019A21
:105210001C7006F0E1F805B0F0BDC0461264FF1F37
:105220004E42FF1F4C42FF1F4A42FF1F1064FF1FE8
:105230000E64FF1F4842FF1F6E64FF1F5042FF1F96
:105240000C64FF1F13B50C4B1C78002C11D10028E7
:1052500001D00A4B18600A4A0A4B11780A4A1078A2
:105260000A4A01920A4A0092002205F001F9200040
:1052700016BD1124FBE7C0466D64FF1F0864FF1FC5
:105280006C64FF1F5C64FF1F6E64FF1F4864FF1F98
:105290004C64FF1F10B5064B12201B78052B06D15E
:1052A000044B13221988044B187801F0EBF910BD58
:1052B0006D64FF1F5042FF1F6E64FF1F10B5002476
:1052C0000122114B52421870104B1C70104B1A8067
:1052D00001F084FF04220F4B21001A700E480C329B
:1052E00006F0EAFA102221000C4806F0E5FA07223F
:1052F0000B4B1C600B4B1C700B4B1C700B4B1A7038
:105300000B4B1C7010BDC0466E64FF1F6D64FF1F09
:105310005042FF1F6C64FF1F5C64FF1F4C64FF1F43
:105320004864FF1F2264FF1F2164FF1F5242FF1FBA
:105330002064FF1FF8B5174C0600257806A8142432
:105340000078052D23D1B41F134FA5B21824BD42F8
:105350001DD88D1FADB2BD4219D8FA256D00AA42E5
:1053600015D21D000D4F0A3DADB2BD420FD80C4CF9
:1053700026800C4C21800C4900240A800B4A1380A3
:10538000FFF714FF0A4B0421187806F035F82000C7
:10539000F8BDC0466D64FF1F790C0000750C00005D
:1053A0004E42FF1F4C42FF1F4A42FF1F4842FF1F51
:1053B0006E64FF1FF0B50BB20D0089B0002B00DB4F
:1053C00070E1A44E307806F0BFFA041E50D0037886
:1053D000A22B00D122E1D02B1AD0912B45D14378BA
:1053E0000E2B42D19C4B82889A423ED19B4A8368C5
:1053F0001278052A39D1032018567F2835D0984BCA
:105400001B68002B31D05B68002B2ED098472CE016
:105410008078072829D806F0CFF90428183F3F7470
:10542000A8D86378002B0CD101218C4B19708D4BBF
:105430001A78002A5BD08C4B307801F035FD0028BB
:1054400055D00722854B1A7051E061780029F8D1B8
:10545000E378002B11D0854A854B1278307801F023
:1054600023FD60706378002BEBD1200006F024F858
:1054700080200002684009B0F0BD784B1B78022BF9
:10548000F3D00121307806F02FF90028EAD101216C
:10549000307805F0E1FFE5E76378002BD1D16F4F5D
:1054A000032807D13B78052B02D101333B701EE066
:1054B0000223FBE76F4B1A886F4B0293002A0BD035
:1054C0001B78002B03D00121307805F085FF3B7855
:1054D000062B04D1013BE9E7029B1A70F7E7042B86
:1054E00041D10121029B3078197005F0B5FF5C4B6A
:1054F0001B68002BB9D01B68002BB6D0574A107818
:1055000084E76378554F002B27D10622211D5B4885
:1055100006F00AFA62895A4B5A491A80A2895A4BF4
:105520001A80E3890B800521397058490A80584A4E
:105530001380228A574B1A80574B1B78012B09D1B5
:105540001F2000F0C3FEFA2292004243042130786B
:1055500005F042FF0022484B75E7312B00D070E781
:105560000022454B1A700323A0E70622002143487E
:1055700006F0A2F90023454A04211380444A3078FA
:105580001380444A138005F037FF0821307805F076
:1055900033FFA379083B5A425341304A0333137017
:1055A000304B1B78002B06D0334B30781A78002A0A
:1055B00006D001F0B7FC0122314B52421A8096E727
:1055C0000121197005F048FFF5E70821307805F052
:1055D00013FF6378002B00D047E72C4B2D4F02932D
:1055E000E388029A04211380294B3078039323899E
:1055F000039A138063893B8006F076F8002800D078
:1056000033E7264B1B68002B00D12EE70399029845
:105610003A88098800881B68984726E74379132B46
:1056200000D022E70389012B0AD11D4B1B78022BE6
:1056300006D10821307805F0DFFEFFF72BFE14E7D6
:10564000052000F043FE08210200307805F0C4FE7A
:105650000BE7C0466E64FF1F051400006D64FF1F5A
:105660000864FF1F7842FF1F5942FF1F4264FF1F5B
:105670002364FF1F4464FF1F4664FF1F1564FF1F60
:105680005042FF1F1C64FF1F1E64FF1F1264FF1F98
:105690001064FF1F0E64FF1F1464FF1F0464FF1FCC
:1056A0000C64FF1F8020C001014200D0E2E6CB075E
:1056B00031D5324B1B78002B1DD0314E05AC3378E1
:1056C000052B1AD1023B23702E4B21001B7823722D
:1056D0002D4B1B7863722D4B187801F089FB002845
:1056E00009D007202A4B30701B68002B03D01B68A1
:1056F000002B00D098470120BCE60E20254B062247
:105700001B7825492370254B1B78637002ABC018AA
:1057100006F00AF9D8E7022308001840194209D018
:10572000174B1B78052B03D11D4B188805F074FF10
:1057300002209FE60424214203D0FFF737FD20001A
:1057400098E6082308001840194200D193E6154B4B
:105750001C78012C03D0022C0DD008208AE6124BB5
:10576000124A134913481B8812880988008800943C
:10577000FFF7E0FDF1E7FFF78DFDEEE74664FF1F61
:105780006D64FF1F5242FF1F2064FF1F6E64FF1FE6
:105790000864FF1F2264FF1F5342FF1F2164FF1F85
:1057A0005042FF1F0C64FF1F4842FF1F4A42FF1F69
:1057B0004C42FF1F4E42FF1F10B502A804880B2069
:1057C000002C10D1496808784978090201430C4837
:1057D000814209D1022119800A4B59881170DB7866
:1057E00000205BB2537010BD074C0A20A142FAD1D1
:1057F00002211980034B998811705B79F0E7C0464C
:105800006E2A00000C62FF1F6F2A0000F7B515001A
:1058100008AA16884A680F4F147852781202224359
:105820000A24BA4214D10122DBB2019200962A0066
:1058300005F024FD041E0BD1074B1B68002B07D07D
:1058400068782A780002104342425041013098475C
:105850002000FEBD022900008064FF1F30B5012535
:1058600003790400BFB02B4225D01449408805F0CD
:1058700071F828420CD0124B01A95B8D00220B80DD
:1058800002234B800F4B5B888B80608802F042F9CB
:105890000D49608805F05EF8C0070CD50B4B01A9D7
:1058A0001B8800220B8002234B80064B9B888B8039
:1058B000608802F02FF93FB030BDC0467864FF1F0A
:1058C0007C42FF1F0C62FF1F7064FF1FD642FF1F48
:1058D00010B5074C0749200004F0F2FF20000649EC
:1058E00004F0EEFF0721054A054804F0ABFF10BDA8
:1058F000FFFF00007864FF1F7064FF1FECBA001107
:105900007C42FF1F10B5024802F086FF10BDC04662
:105910005D5800110200F0B501270A480A4E5118DF
:105920008B1A002B00DCF0BD082415784308684072
:1059300038404000805B013C58406D08002CF5D198
:105940000132EDE7FFFF000006BB0011F0B50025B6
:105950000F269D4200DBF0BD4C5D070944403440FA
:10596000A400A05801357840F3E70000F0B589B0F5
:105970006A460D000B000F27110010351C7801330B
:10598000260024093E40167054700232AB42F5D115
:105990002023024AFFF7DAFF09B0F0BD0CBB00116B
:1059A000F0B54E780B7889B036020C0017000190E4
:1059B0001E43012A61D9954B9E4200D877E00133FE
:1059C0009E421CD1062A17D1CA788B7812021A433C
:1059D0000B791B0413434A7912061A438C4B5A6104
:1059E00000221A705A808B4A5A608B4A9A608B4AFE
:1059F000DA60002009B0F0BD88225205EEE7884B3E
:105A00009E423CD182498B78002B00D0F6E00C2AD4
:105A100031D10F22A3789343E27812021343227903
:105A2000120413436279120613434B60E279A079A2
:105A300012020243207A00041043627A12060243E3
:105A4000CA60E27AA07A1202024376484A8183420F
:105A500008D804236E49142201980B7005F064FFE6
:105A60001420C7E71201D21889235B059A42F0D8A7
:105A700001238B70BDE7022AFAD00523EAE76A4AC0
:105A800001239642E6D1FFF705FC052F0CD9E378F8
:105A9000A2781B021343227912041A4363791B066E
:105AA0001343624A0393136005F076FEA1E7584D55
:105AB0002B78002B9DD1AB78002B00D1A0E02B8957
:105AC00001339BB20093B34200D091E0132AD4D9A2
:105AD000CF7C8B7C3F02122120001F43FFF71AFF6F
:105AE000874200D08EE0002E3DD1E378A2781B02E1
:105AF00013432279E96812041A4363791B0613439E
:105B000003930A228B4212D1FF23A370E370237107
:105B100063716B89002B09D1E37B227C1B02120489
:105B20001343A27B13431B0901336B8100226B8952
:105B3000002B8ED0002A67D1686837013818000B17
:105B40006B6900030390984205D9686105F014FE63
:105B5000EB780133EB7068681022A11C381805F04F
:105B600023FC2E8145E76F89009A7B1E9BB29342EE
:105B70003AD1E278A37812021A43237905A81B04CC
:105B8000134362796C6812061A43EB680092039221
:105B9000211D0C22049305F0C7FE0120260004A954
:105BA00040421036FFF7E2FE013F012F17D1009A65
:105BB0000B232861824200D04CE704221C492000BC
:105BC00005F0F2FB042203A9686805F015FDE968F9
:105BD000039AFF23914200D13CE7F73B3AE73100BB
:105BE000FFF7C4FE1036DFE70923B742A4D831E738
:105BF000009BB34200D9FCE607232BE7022329E7E9
:105C0000032327E7062325E70A2323E7FFFE0000F7
:105C1000F042FF1F00000111FFFF000050485936FD
:105C200001FF0000FFFF001102FF000034F0004000
:105C3000FC42FF1F10B5034C0B000122210000F0B5
:105C40006BFA10BDF55D00110B8870B506000D00F4
:105C50000224162B11D92B000322094900F05CFA0B
:105C6000041E0AD1074B2A881B88191C934200D9AD
:105C7000111C300089B200F0EFFA200070BDC04660
:105C8000215E00119664FF1F10B54A780400013AA6
:105C90000B000220012A07D80A78002A04D0052226
:105CA0002000024900F038FA10BDC0464F5E0011D6
:105CB0000A7810B50B0004000220002A04D0072245
:105CC0002000024900F028FA10BDC046FB5E00111A
:105CD0000A7810B50B0004000220002A04D0092223
:105CE0002000024900F018FA10BDC046615F0011A3
:105CF00010B5034C0B000B22210000F00DFA10BD73
:105D0000915F001110B5034C0B000D22210000F033
:105D100003FA10BD0360001110B5034C0B000F22F5
:105D2000210000F0F9F910BD5D6000110A7810B58E
:105D30000B0004000220002A04D011222000024996
:105D400000F0EAF910BDC0466D600011002310B5E7
:105D50001322190000F0E0F910BD000010B5034C4B
:105D60000B001722210000F0D7F910BDBF60001111
:105D7000002310B51922190000F0CEF910BD000063
:105D800010B5034C0B001B22210000F0C5F910BD1B
:105D9000F9600011F7B584890D0006000121002C7F
:105DA00022D000238268D3561778002B1EDA0C2CE1
:105DB0001AD90C3CA4B2131940880093230002F0B6
:105DC00086FE431E984101307B06DB0F6B703F233C
:105DD000013C1F40A4B22870AF70AC80002C07D0EB
:105DE000B3680133AB6000210800FEBD0020EBE783
:105DF000AC60F8E70B7803704B8843704B881B0A44
:105E000083700B79C370042070470420022B06D1E5
:105E10000020537811781B02009A0B4313807047BF
:105E20000B8803700B881B0A437002207047042004
:105E3000009983420AD1537810781B0203430B80E8
:105E4000D37890781B02034300204B807047F8B54D
:105E50000D004B7801240021461C03702B788B42E7
:105E600001D82000F8BD6B78B01C4F1C012B10D15D
:105E7000890069184B88022233704B88B9001B0ACD
:105E80007370691805F088FB04360434A4B2F9B2C3
:105E9000E4E7122359436B185A88043132705B8847
:105EA00010221B0A7370691805F076FB1236123443
:105EB000ECE770B5049D14001E00052B01D80420EA
:105EC00070BD637812781B0213432B80E378A278AD
:105ED0001B02134302226B802A71211D681D063E9E
:105EE00005F05AFBB2B22A81E92AE8D82800A11DA0
:105EF0000A3005F051FB0020E2E7002310B50A78D4
:105F00009A4201D8900010BD9A008A185488013333
:105F100004705488DBB2240A447094888470928898
:105F2000120AC2700430EAE710B51100029C062B79
:105F300004D004201022142B01D010BD02222271A3
:105F40004B7808781B0203432380CB7888781B02A8
:105F5000034363800431601D05F01EFB0020ECE765
:105F600010B50C788B7804315C43E4B203702200E6
:105F7000013005F011FB601C10BD0420022B06D17E
:105F80000020537811781B02009A0B43138070474E
:105F900010B50C000A88023105F0FEFA208810BD09
:105FA00070B504000D0004981100012B01D80420E5
:105FB00070BD167852781202324302800200F1322C
:105FC00055701470E125002C00D10C35023B9AB2BB
:105FD0004280AA42EBD80231043005F0DDFA0020FD
:105FE000E6E70420009983420AD1537810781B0217
:105FF00003430B80D37890781B02034300204B802F
:10600000704710B50C000A88023105F0C5FA2088E7
:1060100010BD000070B501211E000420049C0E403C
:106020000B4218D1CB40DDB28D4214D90A49DBB204
:10603000098899420FD32300EE331D7033005800B6
:1060400011184978165C0902314301332152D9B243
:106050008D42F4D8002070BD0843FF1F10B50C001E
:106060000A88023105F098FA208810BD10B50C7826
:106070008B7804315C43E4B203702200013005F0F8
:106080008BFA601C10BD10B511000298032B01D8CB
:10609000042010BD14785278043B1202224302807F
:1060A000CA788C781202224342809AB28280EB2A0C
:1060B000EED80431063005F06FFA0020E9E710B59C
:1060C0000C000B8803700B881B0A43704B8883708D
:1060D0004B881B0AC3708A880430063105F05CFACD
:1060E000A088043080B210BD0420012B03D1002011
:1060F0001378009A1370704710B50C000B8803706A
:106100000B881B0A43704A880230043105F044FAB8
:106110006088023080B210BDF0B589B003931E4B89
:10612000029242000700D05A019102F020F8132594
:10613000061E2DD0029B01240370019B002B04D06E
:10614000001903999847001984B26B461B7A5BB219
:10615000002B0FDA1021380002F01CFB1925002853
:1061600013D130003219E1B202F066FC051E0CD1E9
:106170000C34A4B2042304AA380005A9938006961F
:10618000948101F0AFFD051E02D0300005F094FAB5
:10619000280009B0F0BDC0469464FF1F70B505002B
:1061A0000C0000280CD00020814209D010222000D1
:1061B000044905F0F1F901202B7823736B786373A0
:1061C00070BDC0464CBB0011F0B506000D001700B5
:1061D0001C0085B002291BD00020102907D1022BFA
:1061E00007D0102B03D115E00020102C08D005B0EB
:1061F000F0BD69463800FFF7D1FF2A0069460BE081
:1062000069463000FFF7CAFF22006946380004E003
:10621000022BE9D12A003900300005F02DFAE6E71B
:10622000031CF02800D9F023032008499AB2013A50
:106230000B80D317034006499B189B100B80D30F8C
:1062400004499B185B100B807047C0460C43FF1F2E
:106250000A43FF1F0843FF1F034B1B888B4202D3D7
:10626000024B4000C15270470C43FF1F9464FF1F54
:10627000014B4000185A70479464FF1F1722014BCE
:106280001A8070479464FF1F70B505000E2005F05A
:106290001BFB041E13D0D02303700023062283703F
:1062A00007494570033005F077F9064B2100DA8A7B
:1062B00062811B7E2373044B187805F045F970BD8D
:1062C000B064FF1FA064FF1F5C43FF1F262803D894
:1062D000024B4000C05A70470148FCE70E43FF1FC5
:1062E000FFFF000070B506000C00094D1C220021C4
:1062F000280005F0E1FA074B1E70074B1C7005F0F3
:1063000093FA0123002801D0002312202B7070BDC6
:10631000A064FF1F5C43FF1FC164FF1F70B5050031
:106320000D4C0800E260A16010220021656005F0BC
:10633000EBFA012803D11021A06802F058FD1022C9
:106340000021280005F0E0FA012803D1102160683F
:1063500002F04DFD70BDC046A064FF1F70B5041E65
:1063600005D1002903D006220D4805F015F90D4B83
:106370001D78012D11D1002C05D102221A7005F0D3
:10638000F3F9280070BD00221A70074B1B78FF2B11
:10639000F7D02000FFF778FFF3E70025F1E7C046CC
:1063A000B064FF1FA064FF1F5C43FF1F030010B514
:1063B000002801D1002010BD00780B4A002803D12D
:1063C0005988D1821B7913761378022BF2D10023DE
:1063D000984200D103331370044B1B78FF2B01D07C
:1063E000FFF752FF0120E6E7A064FF1F5C43FF1F99
:1063F000002911D000280CD04B79012803D140226C
:106400005242134303E03F221340032802D00120ED
:106410004B7170474022F4E70800FAE770B5094D68
:106420000100287800280BD0074C0622200005F038
:10643000B3F821002878FFF7DBFF200005F024F8EF
:1064400070BDC046C064FF1F9A64FF1F00290AD0B8
:10645000012808D13F224B799343C02B03D0403B06
:106460005A425341981C704770B5174D06002B785F
:10647000FF2B15D00A2005F027FA041E10D0D023D8
:106480000370C83B8370114B11491B784670C37071
:106490000622043005F080F82100287805F054F831
:1064A0000C4B1B78012B0DD10B4B1B68002B03D021
:1064B0009B68002B00D09847084B04211878084AA5
:1064C00005F0CAF870BDC0465C43FF1FC064FF1FE3
:1064D0009A64FF1FBC64FF1FE864FF1FEC64FF1F8A
:1064E00060EA0000014B98687047C046A064FF1F37
:1064F000014BDB6818687047A064FF1F074B10B59D
:10650000DA68136801331360054B1878FF2803D04D
:106510008021C90104F0A0FF10BDC046A064FF1F88
:106520005C43FF1FF7B50E0002F0C8F8051E1CD033
:106530000E4B06621F78002F00D10778AB79102030
:10654000019305F0C1F9041E0FD0D0230380C73B8F
:106550008370019BE91DC3700622043005F01CF80E
:1065600021003800E66004F0EFFFF7BD5A43FF1F3B
:10657000014B18787047C046C064FF1F054B0028C8
:1065800005D1054B1A78054B002A00D1014B1800A4
:106590007047C046B064FF1FC064FF1F9A64FF1FAE
:1065A000014B58687047C046A064FF1F024B186833
:1065B000431E9841C0B27047C464FF1F421E0300CF
:1065C0000120152A03D9FF3B5A425341D8B27047E4
:1065D000F0B51C0000230E0085B0039002920B70F2
:1065E000029A934201D3002019E0E55C5A1CD2B212
:1065F000002DF8D0029851198142F4DC0233DFB249
:10660000A35C18000193FFF7D9FF002807D0013DD4
:10661000019A0399EBB233708A4202D1E01905B0B6
:10662000F0BDDB19DBB2DBE710B50C0002F09EF821
:1066300003001220002B03D02100588805F024F914
:1066400010BD000070B50E4D84006359002B15D0AD
:10665000186A002801D005F027F92B59586A00283C
:1066600001D005F021F92B59986A002801D005F0D6
:106670001BF9285905F018F900232B5170BDC046AD
:10668000D064FF1F1C4B70B504000E00150099422A
:106690000AD11A4B1B68002B01D1122070BD1B6858
:1066A000002BFAD09847F9E7154B994215D1134BB7
:1066B0001B68002B0AD01B68002B07D098470028C6
:1066C00004D1104B1C70104B1D70E7E7290020000F
:1066D000FFF7AAFF0028E1D1F3E7080001F0EEFF81
:1066E0000028DAD003780320A342D7D12900300054
:1066F00005F0CAF8D2E7C046FEFF0000CC64FF1FD9
:10670000FFFF0000C964FF1FC864FF1FF7B5040046
:10671000808801F0D3FF0025A84203D00578A08827
:1067200002F008F81C4E3378002B1FD0AB421DD16D
:106730001A4B28001978FFF777FF002818D000239C
:106740003370A3790820A778A688019305F0BCF8D8
:10675000011E0DD0D0230370CA3B8370019B47708C
:1067600086808371280004F0EFFE01E0002DE8D15F
:10677000A0880B4B8200D358002B01D0FFF762FF9B
:106780001721A088FFF768FDA08801F027FDA088E9
:1067900001F0FEFDF7BDC046C964FF1FC864FF1FBE
:1067A000D064FF1FF0B587B01D000CAB1B8807003D
:1067B00001930DAB1B88142002930EAB1B881600AF
:1067C00003930FAB1B880091049310AB1B880593B8
:1067D00005F07AF8041E1AD0D0230370CB3B477023
:1067E0008370C670062229000430002D11D004F0F9
:1067F000D3FE019B21006381029B0098A381039B30
:10680000E381049B2382059BA37404F09DFE07B0E3
:10681000F0BD05F051F8ECE7F7B5009308AB1B8825
:1068200007000C200D001600019305F04DF8041E22
:1068300013D0280001F042FF00280FD00078D023A9
:106840002370C93BA370009B21002381019B6770CB
:10685000A580E680638104F077FEF7BD014B1878D0
:10686000EDE7C0465C43FF1F13B50400648903894C
:10687000C2888188C0780094FFF7CEFF13BD000066
:1068800010B5044C2068002803D005F00DF8002353
:10689000236010BDD464FF1FA122F0B5818892004F
:1068A0004A43384B384F1B6804009B189D229200C6
:1068B0009B18827989B01A603B68002B5FD01D78E5
:1068C000324B1B68002B04D05B68002B01D00020EA
:1068D0009847260008363100E079FFF7B7FD237DA1
:1068E000E0710200E0780493638A29000393238A0D
:1068F0000293E3890193A38800933300FFF752FFCB
:10690000E378002B0BD1E289A379A188029201964A
:10691000E27928000092012201F0DAFEE0703B6883
:10692000002B20D0FFF7ACFF194D287800281AD093
:10693000184B1978FFF778FE002814D02B78E678EA
:1069400008200793A78804F0BFFF011E09D0D023B9
:106950000370CA3B4670837087808671079804F085
:10696000F3FD00232B701721A088FFF775FCA0888A
:1069700001F034FCA08801F00BFD09B0F0BD064B1E
:106980009DE7C0463409FF1FD464FF1FE864FF1F62
:10699000C964FF1FC864FF1F5C43FF1FF8B50700F1
:1069A00008000E0001F08AFE041E18D02620FFF712
:1069B0008DFC051E00D12578062004F085FF041EFD
:1069C0000DD00021062204F077FFD0232370C23BB4
:1069D00021006770A370A680E8B204F0B5FDF8BD91
:1069E000F0B585B001930AAB1B78070002930BAB9F
:1069F0001B7808000D000092039301F05FFE061E55
:106A000022D0102004F060FF041E1DD010220021AF
:106A100004F052FF2620FFF759FC002800D13078FF
:106A2000D0232370C13BA370009B21002372019BE4
:106A300067706372029BA580A372039BC0B2E3726E
:106A40000C9BE36004F080FD05B0F0BDF7B50D00D0
:106A5000019001F033FE071E20D00E2004F034FF19
:106A6000041E1BD02620FFF731FC061E00D13E7805
:106A7000D0232380C53B0622A370F91DE01C04F03F
:106A80008BFD019B2A0063810123DD401A401D40DC
:106A9000210022736573F0B204F056FDF7BD0000CB
:106AA000F0B585B0029010000D0017000A9E039308
:106AB00001F004FE041E31D0029B002B2ED1039B5B
:106AC00002795B0724D5122313430422002E08D138
:106AD0000B99002905D10C99002902D10D990029A3
:106AE0001AD01A430D9B2271002B00D0C9E0002E52
:106AF00000D1CFE0002D00D0CCE0606A002801D0AA
:106B000004F0D2FE1C21300004F0B6FE606205E005
:106B100002239A430E33D7E793432371654BBA00A0
:106B2000D458002C00D1AAE0002E10D0236A002BEC
:106B300003D11C2004F080FD20625E4BBA00D358C4
:106B4000186A002803D01C22310004F025FD0C9B9C
:106B5000002B12D0574CBB001D596B6A002B03D180
:106B6000162004F069FD6862BB00E358586A0028EB
:106B700003D016220C9904F00FFD0D9B002B11D0B1
:106B80004C4DBC006659B36A002B03D1142004F0AD
:106B900053FDB0622B59986A002803D014220D9936
:106BA00004F0FAFC380001F089FD051E67D0414B66
:106BB000BA00D358002B62D01A6A3420002A00D1C0
:106BC0001C389A6A002A01D0143080B20B9A002A2D
:106BD00001D01C3080B25B6A002B01D0163080B22D
:106BE00004F072FE041E4AD01822002104F064FE54
:106BF0002620FFF76BFB0190002801D12B78019331
:106C0000D0232370029B200063700A23294EA370B7
:106C1000039BBD00A371AB59A780196A18300029E6
:106C200005D01C22A06004F0B7FC2000343073595A
:106C3000996A002907D0030014221433E0600293FC
:106C400004F0AAFC02980B9B002B08D003001C2226
:106C50001C330B992061029304F09EFC0298735937
:106C6000596A002903D01622606104F095FC6B4636
:106C70002100187904F068FC3800FFF7E3FC05B048
:106C8000F0BD10220D9B0D991B69A018236204F022
:106C900083FC2CE70B9B002B00D13FE7012D00D09C
:106CA0003CE7606A002801D004F0FEFD1C210B982F
:106CB0002AE7C046D064FF1F10B5044C20680028A6
:106CC00003D004F0F1FD0023236010BDC464FF1F56
:106CD0000B4B07B51A68002A01D100200EBD69468A
:106CE000531C012012780731FFF772FC0028F4D002
:106CF00002780123100018401A42EED0EEE7C04699
:106D0000E064FF1FF0B51F4F01203B6887B0002BE8
:106D100025D09B78059300F0B3FB002821D00A20F2
:106D2000FFF7D4FA04000B20FFF7D0FA164B05004A
:106D30001E78731E9E413B68F6B2191DD878FFF786
:106D400057FB3B682900DA7A043303929A7901935E
:106D50000292009033002000059A04F0D5FC07B0A1
:106D6000F0BDFFF7B5FF002805D00620FFF7AEFA0B
:106D700004000720D8E70820FFF7A8FA040009203C
:106D8000D2E7C046C464FF1FC064FF1F70B50A4E3F
:106D9000040033780D00FF2B0DD0042004F094FD87
:106DA000011E08D0D0230370CE3B45708370C470A1
:106DB000307804F0C9FB70BD6C43FF1F70B5040050
:106DC00006200D0004F080FD011E0AD0D0230370C0
:106DD000CD3B8370054B44701B688580187804F0A8
:106DE000B3FB002C01D0FFF767FF70BDC464FF1F29
:106DF000F8B5264F06003B680D001124002B05D185
:106E00000522234B1B78134202D112242000F8BD27
:106E1000204A10241268002AF8D01278002AF5D0EF
:106E2000DB0719D52B789A1E012A1AD80C2004F0FA
:106E300003FC132438600028E8D000230A224370A2
:106E400029000670023004F0A7FBFFF75BFF041E69
:106E50000AD0FFF731FFD9E700F012FB0028E1D19B
:106E6000E4E7002BE2D0D0E70B4B1B78032BCDD10E
:106E70001D20FFF72BFA094B18800028C6D0084BBD
:106E800004211878074A04F0E7FBBFE7C464FF1F3A
:106E9000C164FF1FE064FF1FC064FF1FBE64FF1FCB
:106EA000EC64FF1F60EA0000F7B50193194B140072
:106EB0001A78052306000F0012201A4221D001295A
:106EC00020D1154B1D68002D1BD002201F2C18D877
:106ED000002C02D0019B002B13D0104B1F221E70E0
:106EE0006E1C0021300004F0E7FC01992200300004
:106EF00004F052FB310020002C70002F06D004F06B
:106F00006BFCFEBD064B12201D68DCE704F054FB51
:106F1000F7E7C046C164FF1FE064FF1F6C43FF1F1B
:106F2000DC64FF1FF8B50F4E12243368002B17D016
:106F30001B780F3C834213D100250B4F0221387878
:106F400004F05AFA094B042138781D8004F054FAF1
:106F5000074B28001D8033685C7004F0DDFA0400E4
:106F60002000F8BDC464FF1FEC64FF1FD864FF1F3E
:106F7000BE64FF1F70B5012823D11B4C2388002B52
:106F800003D01A4A1578002D07D0194B1B68002B27
:106F900002D01878FFF7C6FF70BD3B2B02D93C3BEF
:106FA0002380F9E7134E0221307804F025FAFA2203
:106FB0002388920002215A43307804F00DFA25808C
:106FC000EAE70B4B1B68002BE6D00B4B1B785B07EB
:106FD000E2D5084B0221187804F00EFA0022024B89
:106FE0001A80FFF769FED7E7D864FF1FBC64FF1F54
:106FF000C464FF1FEC64FF1FC164FF1FF8B51E4D82
:107000002868002803D004F04FFC00232B601B4E9F
:107010003068002803D004F047FC00233360184F89
:1070200005243B7818002040234221D0154800F069
:107030002BFA3B78234213D0202004F0FDFA28607D
:10704000002813D02022002104F036FC202004F078
:10705000F3FA041E306005D02022002104F02CFC3D
:10706000002004E0286804F01FFC2C601320F8BD09
:1070700000F00AFAF4E7C046E064FF1FDC64FF1F7B
:10708000C164FF1F6043FF1F10B50A4C23681A1E1E
:107090000ED0002808D10130587004F03DFA0028C5
:1070A00005D02368002B02D00021FFF787FE0122C4
:1070B000100010BDC464FF1FF7B5274E05003368EC
:1070C0000191181E21D05C78244F012C30D1FFF79C
:1070D000FFFD002825D02000FFF7F8F80400412824
:1070E00014D91F4B022118781E4A04F0B5FA1E4B22
:1070F0003C3C1C80022233685A703B78002B14D130
:1071000028000199FFF75AFE0120FEBDFA229200E5
:107110004243002AEED0124B0221187804F05CF9A9
:10712000E8E7FFF7D3F80200F3E700233B70EBE753
:107130003B78002BE8D1032004F0C6FB011E08D0E9
:10714000D0230370CC3B457083703368187804F00B
:10715000FBF9FFF7B1FDD7E7C464FF1FBC64FF1F55
:10716000EC64FF1F60EA0000D864FF1F10B51749E8
:10717000838802008B4220D011D815498B4217D04A
:10718000144900205B1899B2012907D89268117838
:107190005A425341D8B2FFF7F9FD012010BD0E4A03
:1071A00000209B1807229BB29A424041C0B2F5E7EB
:1071B00083681878FFF768FFF0E7836899785A7852
:1071C000090218781143FFF777FFE7E70A2000006C
:1071D00006200000F8DFFFFFAFDFFFFF014B187054
:1071E0007047C0466D43FF1F10B5064C207001F07C
:1071F00041FA207804F0F8F90521207800F062FDCA
:1072000010BDC046EC64FF1F0BB273B50D00002B20
:1072100000DBC4E0884B187804F096FB041E0ED007
:107220000378912B0FD0A22B00D1A1E0834B1878CB
:10723000FF2852D0210004F087F900284DD180208A
:107240000002684076BD43780F2B76D013D8052B0B
:1072500070D00E2BEAD18088794B98422BD8794B8D
:1072600098421BD8784B9842E0D1A3681878591CF3
:10727000FFF774F838E03E2BD8D18378032B74D015
:107280006CD8012B6ED0022BD0D1704B1B68002B19
:1072900023D05B68002B20D098471EE06C4BC018B1
:1072A0000C28C3D804F0C0F81DC2C2150BC20B0BCA
:1072B0000B3223C23C00674BC0180728B6D8664B78
:1072C0001B68002B09D01B68002B06D020009847B4
:1072D0000AE0A3681878FFF7C7F8200004F0ECF87C
:1072E000ADE7A068FFF762F800289FD0F5E7A36834
:1072F0001B78002BF1D0554B1B68002BEDD01B6881
:10730000002BEAD0210055489847EDE74F4B1B680A
:10731000002BE2D01B68002BDFD021005048F3E7A0
:10732000504B1B68002BD8D05B68002BD5D02100B8
:107330004348E9E7FFF7EAF9CFE780884A4B9842EC
:1073400003D04A4B984200D070E7464B1B68002B95
:10735000C3D05B68002BC0D02100D5E7153B012BC3
:10736000BBD963E7FFF798FAB7E7FFF77DFAB4E711
:107370003F4B1B78042B07D100236A461380017909
:10738000408800F0C5FCA8E7364B1B68002BA4D052
:107390005B68002BA1D00100364898479DE7012487
:1073A00021420AD0294B1B68002B04D05B68002BBC
:1073B00001D000209847012043E78B070AD5264BD0
:1073C0001B68002B04D05B68002B01D0200098477D
:1073D000022036E70421280008400D4200D131E7A1
:1073E000254E3388002B21D0013B9BB23380002BEC
:1073F0001AD1FFF7DBF800280AD0204B1C70164B7F
:107400001B68002B04D05B68002B01D0200098473C
:10741000FFF7C6F8694601F001FD6846FEF7FEFF7A
:107420001D20FEF753FF308004200AE7024B187836
:1074300003F0E2FFF8E7C046EC64FF1F6D43FF1F57
:107440000E2000000120000009100000E464FF1F6E
:10745000FEDFFFFFAFDFFFFFE864FF1F0C2000002F
:107460000B200000CC64FF1F0D2000001320000043
:10747000C164FF1FFFFF0000BE64FF1FBC64FF1F4D
:1074800010B501F09BF910BD014B18607047C04664
:10749000E864FF1F0B880020162B01D81723042057
:1074A000014A13807047C0469664FF1F0020704752
:1074B000074A03001188814207D091880020994231
:1074C00002D101308000101870470020FAE7C04652
:1074D000F464FF1FF0B58F7806000D00C5B01E2FB5
:1074E00015D1FFF7E5FF051E03D10024200045B0AC
:1074F000F0BD00223B003100C078009200F0B2FBEA
:107500000400A81C00F0D2FBFF23EB70EEE7264B33
:10751000062403931B78FF2BE8D0182FE6D87B08AE
:10752000224A013BDB0002929A589446002ADDD0A1
:10753000029AD3185B68002BD8D00878002802D1B3
:107540004B78012B02D10624122FCFD107AFAB8885
:10755000697800976446AA68A047041EC6D1AB7834
:10756000029A5B08013BDB00D318390030005B68EE
:107570009847041E0BD1AB78042BB6D0039A310088
:1075800010782200009700F06DFB0400AEE76A78E7
:10759000002AABD1AA7805A93B88087130000A708F
:1075A0004B80FEF747FBA0E77043FF1F5CBB001159
:1075B0001D4B37B5050098420BD000290AD1FFF7C3
:1075C00077FF002805D11948FFF772FF002800D087
:1075D000058037BD01291AD1FFF76AFF041EF8D0D4
:1075E00001235B420380A378FF2BF2D0FE2B07D050
:1075F0000023E0781422009329001E3300F032FBB0
:10760000A01C00F053FB01235B426380E1E70229E9
:10761000DFD1013901F0BEF80028DAD12800FFF7E8
:1076200047FF041EDFD1D4E7FEFF0000FFFF00008C
:10763000022210B5074B52421A80074801325A8085
:107640009A80DA8000F07EFA044801F025F80020E4
:1076500010BDC046F464FF1FD5740011B175001150
:107660000388F7B50400002B02D102252800FEBDD7
:1076700042680221137825485268FEF7A5FD0028CC
:107680002ED0234F01253A88002AEFD0802321886D
:107690005B0201259B1A9942E8DC0C2003F0CCFF29
:1076A000061E31D03B8822889C4600231800019595
:1076B00061469DB2491989B2AA421BD8002801D05F
:1076C00062443A8000233000082208C0210003F001
:1076D00063FF104A1368002B13D100251660C5E71D
:1076E0006268022113780C485268FEF76DFD00288D
:1076F000C7D1BAE760681D01401941810133019883
:10770000D6E71A001B68E6E71325AFE7CABB0011EE
:107710006E43FF1FF064FF1FC8BB0011014B1870C0
:107720007047C0467043FF1F14230A0010B51A406B
:10773000194204D00122102101F048F810BD4B0677
:10774000F9D4012088434000F8E710B514008B06F7
:1077500004D50122102101F039F810BD08230A00D8
:107760001A40194202D14BB2002B0FDA102101F05E
:107770002DF8002808D02300F2331B78002BECD022
:10778000F1342378012BE8D10020E6E703208907B4
:10779000FAD4E2E7F0B51F00184B85B01C680190E1
:1077A00002910392002C27D1200005B0F0BDA568FE
:1077B0003301ED186B89019A934211D3029A9342D7
:1077C0000ED8002F04D10A9B002B10D12C00EBE720
:1077D0003B002978039A6868FEF7F6FC0028F2D18E
:1077E0000136B6B2A388B342E1D82468DAE7A368C9
:1077F0000A9A5B891380E9E70026F3E7F064FF1F2C
:1078000037B50C000A8849880123914217D3002A12
:1078100015D0651D23792A0002210A48FEF7D4FC01
:10782000102300280BD023796188208800242A00A7
:107830000094FFF7AFFF0A23A04200D023001800F6
:107840003EBDC046CABB001113B50A00088849886E
:10785000012388420BD8002809D00024137905326F
:107860000094FFF797FF0A23A04200D023001800DE
:1078700016BD13B50A0008884988012388420BD831
:10788000002809D00024137905320094FFF782FF05
:107890000A23A04200D02300180016BDF0B58BB01B
:1078A00003904A8808880E000123824255D300289D
:1078B00053D00023012704AC2370002271881300E9
:1078C0000092FFF767FF051E3ED02078002835D1D3
:1078D0002B78022B18D167706A8983000130E31876
:1078E00080005A8069680222201803F055FE237830
:1078F0000133DBB22370042B19D93B0068890130B6
:1079000080B2002BD9D01FE00223637012235843AA
:107910006A89231804305A8069681022201803F0FD
:107920003BFE23780133DBB22370002BE5D10C4AF8
:107930006B899B185A425341DBB2DFE76378012B16
:10794000E4D12B78022BC7D022780A23002A04D056
:1079500021000398FEF798F9002318000BB0F0BD42
:107960000100FFFF0F4BF0B504001868002816D087
:1079700083685D89A54207D88288AE18B44203DACD
:1079800012019A18934201D10068EFE71E005F8947
:107990001036A74204D1002900D00D801800F0BD98
:1079A0003300EFE7F064FF1F70B505000C00088896
:1079B0000021FFF7D7FF03000120002B04D0220095
:1079C0002800197AFFF7C1FE70BDF7B50C0000253D
:1079D00001902300EE331B78AB4201D800200AE06F
:1079E0006B00E65A00213000E718FFF7BBFF0028C4
:1079F00002D126800130FEBD017A0198FFF794FE86
:107A0000002802D03B882380F5E70135EDB2E0E79E
:107A100010B5040008880021FFF7A4FF030001202F
:107A2000002B03D02000197AFFF77EFE10BD000066
:107A3000054B1B68002B01D1180004E09A6852899D
:107A40008242F6D198887047F064FF1FF0B50E2788
:107A5000002687B0039302ABFF183E8005001F4B42
:107A600040891400984207D02B78013000976A684B
:107A700080B2FFF78FFE060002212B7818486A6853
:107A8000FEF7A2FB00280FD06C892000FFF7D0FF83
:107A9000002802D0013C0419A4B2039B002B00D0A3
:107AA0001C80300007B0F0BD02212B780D486A68B9
:107AB000FEF78AFB0028E7D102212B780A486A6882
:107AC000FEF782FB002807D0002EDED03B88A342C1
:107AD000DBD17489013CDFE76C89DEE7FFFF000042
:107AE000CABB0011C8BB0011C6BB001110B50C0009
:107AF000FFF7DEFC03000220002B0AD0002C00D090
:107B000023609B781720FE2B03D00138FF2B00D178
:107B1000002010BD73B50D0001A904001600FFF789
:107B2000E5FF172805D0002E04D129002000FEF71C
:107B300027F976BD01221021200000F047FE002821
:107B4000F3D0F6E7014B18607047C0460065FF1F91
:107B500037B56B469D1D010004000222280003F08A
:107B6000E3FE2B88B02B0ED12379122B09D12300F1
:107B7000FA331B78012B06D10121608800F0E0F870
:107B800001E01B2BF8D037BD10B5054B0421187050
:107B900000F098F8FFF74CFDFEF770FB10BDC046F3
:107BA0000465FF1F0020F0B50BB20F0087B08342C1
:107BB00034DA274B187803F0C7FE051E2BD0037864
:107BC000A02B25D103AE3100FEF7E4F8041E0BD143
:107BD000B378DB0724D51F4B06341B68002B03D07A
:107BE0003100688898470400A868002801D003F095
:107BF00063FD002C08D1184A039B1340174A934297
:107C000006D0B3781B2B03D00121688800F098F8C8
:107C1000280003F051FC80200002784007B0F0BD3E
:107C20000F4B1B68002B10D0310068889847041E4A
:107C3000DAD07378002BD7D1B27801A90A704B80C3
:107C40000C716888FDF7F6FFCEE70624F1E7C04621
:107C50000465FF1FFC64FF1F00FFFF00000112000E
:107C60000065FF1FF7B50190FC200D0017001E00F6
:107C700003F02AFE04001320002C12D0B0232000B1
:107C80002370089BF4226770658026710830002BF2
:107C900008D0190003F080FC2100019803F054FC87
:107CA0000020FEBD089903F007FEF5E710B5041E9D
:107CB00006D00078FD2803D803F0F6FBFF232370DD
:107CC00010BD00000A1F93B210B504000220032B60
:107CD00005D882400020024BD1529B189C7010BDE9
:107CE0002465FF1F0B8870B5043B04000D000220C3
:107CF000032B0BD80121200000F04CFD03001420C1
:107D0000002B03D02900200000F0DEFB70BD000036
:107D100007B51300034A00920A00012100F02CFC71
:107D20000EBDC0464D7F001107B50192032200929F
:107D3000024B0A00122100F049FC0EBDCB7F00115E
:107D400007B56B4601AA11800449D880087806332C
:107D5000012802D1190003F09FFD07BD0565FF1F33
:107D60000C4B10B518700023FF210B4A13801381B0
:107D700093819380094A5380137051729381937257
:107D8000D174D3821375517703F09EFC00F0FCF997
:107D900010BDC0463465FF1F2465FF1F0665FF1F29
:107DA000F0B58DB06B46002003910C229B5E8342A0
:107DB00000DBB0E05D4B187803F0C6FD051E00D176
:107DC000A4E00378902B00D09DE006AF0100468828
:107DD000380000F013FA79680400002900D19CE013
:107DE0003B88052B6ED13B89032B1CD905AC2000A9
:107DF00000F0A2F86288172A61D83989131D9942C8
:107E000031D17968237804310291D90738D5607867
:107E100000F08EF9071E06D0002303712378012B92
:107E200008D0132B23D0A868002800D178E003F0F5
:107E300043FC75E06288029909A800F0A6F8029058
:107E4000380000F08BF909AA2378387A01920022D1
:107E500031000092029A00F012F9380000F064F943
:107E6000029B002BDFD0300000F080F9DBE70378C5
:107E7000032BD8D16288029909A800F0D6F8DEE772
:107E8000122B13D1029909A800F0B5F8021EEAD10D
:107E900027498B88002BC6D0887909A923780191BE
:107EA00061780091310000F0EAF8BCE7002302AAF3
:107EB00093833000617809AAFFF72AFFB3E71D4BCF
:107EC0000993F6E7042B02D09A1F012AABD8184A6F
:107ED000043B9B00995A0029A5D0D2189078310014
:107EE0003A0000F0AEF800289DD13B88042B03D067
:107EF00001213000FFF724FF012C04D1A8680028DD
:107F000001D003F0D9FB280003F0D6FA8020039BB0
:107F10000002434018000DB0F0BD012800D182E7F7
:107F200001213000FFF70CFFEDE7C0463465FF1F6D
:107F30002465FF1F010017000B7803704B78437016
:107F4000CB788A781B021343438070470A8803006A
:107F500002700A88120A42700A88012A06D14A88E9
:107F600082704A88120AC27004207047022082423E
:107F7000FBD14A8804309A704A88120ADA708A88DB
:107F80001A718A88120A5A71EFE710B504000120AD
:107F900082420CD94B780A781B0213432380834218
:107FA00006D1CB788A781B0213436380002010BD72
:107FB000022BFBD1CB788A781B02134363804B7969
:107FC0000A791B021343A380F0E70B8803700B8828
:107FD0001B0A43704B8883704B881B0AC3708B88C5
:107FE00003718B881B0A4371CB888371CB881B0A72
:107FF000C3710820704703000120082A14D14A7871
:108000000878120202431A80CA7888781202024362
:108010005A804A790879120202439A80CA7988798B
:10802000120202430020DA80704710B504000120DC
:10803000022A05D100204B780A781B0213432380C3
:1080400010BDF8B5060010200F00150003F03CFC31
:1080500004000120002C0ED0A0230C222900238034
:108060006780201D002D07D003F096FA2100300014
:1080700003F06AFA0020F8BD03F01EFCF6E7F7B53E
:108080001E00009008AB142017001D78019103F02A
:108090001BFC041E12D0A2230370019B4770438077
:1080A000099B057146710C220830002B07D019007E
:1080B00003F072FA2100009803F046FAF7BD09991F
:1080C00003F0FAFBF6E737B5041E0FD04388002B08
:1080D0000CD00025C1881323007A17220195009542
:1080E000FFF7CDFFFF2365806372257037BD000069
:1080F00010B50C4904004A88002A09D08B89002B4E
:1081000005D00020CB8A0222834201D010BD01227B
:1081100013000A20434300204032C854C81842804C
:108120000472F3E70665FF1F002343800370704766
:10813000094B00211A0010B55C88002C06D01C7970
:10814000844203D10A234B43D01810BD01310A33B6
:108150000329F1D10020F8E70665FF1F10B50400E0
:10816000407A03F0A1F9FF23637210BD7047043019
:1081700010B580B203F0E8FA002803D00421494288
:1081800003F012FA10BD000070B50025104CA06875
:108190002580A581A580A84202D003F08DFAA560B4
:1081A00000250C4C0C4B606D1D80230058331D7056
:1081B000A84202D003F080FA6565002560680028B7
:1081C00001D003F079FA013508340A2DF6D170BDDB
:1081D000CC65FF1F7065FF1FC065FF1F70B5041ED3
:1081E00009D1054D2880A881A880A868002802D060
:1081F00003F062FAAC6070BDCC65FF1FF0B54B8830
:1082000085B00193002343600A7905000F00022A1C
:1082100000D07BE0CA88032A17D98B685E7819786A
:108220003602DC78D8790E4399781B7A24021B0237
:108230000C43034353495BBA0B80331D93421ED159
:10824000042C04D0631F022B0ED9012015E0019AE3
:108250004D4B1201D35A002B06D00198FFF7BEFFF9
:108260004A4A1369013313610421B8682E812C80B6
:10827000494203F099F96860002005B0F0BD434D14
:10828000042C06D0631F022B0FD9EB680133EB607F
:10829000DBE7019A3C4B1201D35A002B05D0019821
:1082A000FFF79CFF2B6901332B61374B30000293A2
:1082B000019B029A1B010193002301998C468B526A
:1082C000130063449C8003939E81FFF750FF039B40
:1082D000041E986016D00421B868494203F064F97E
:1082E000FA880100043A200003F056F90199029A35
:1082F000FB888A5A043B9B18029A8B522B680133E5
:108300002B60A2E7AB690133AB619EE71E4B029382
:10831000019B1E01029BF35A002B2DD002998C1950
:10832000A068002828D0012A26D1FA889B189BB281
:108330007352A189994217D39B1AC018B96803F0E8
:108340002BF9029BA289F35A934200D07DE70022C9
:108350002B81A3882B80A3686B60029BF2520B4A8F
:1083600053680133536070E7084A936801339360A0
:108370000198FFF733FF68E7044A536901335361FB
:10838000F6E7C0463665FF1FCC65FF1F3C65FF1F43
:1083900070B5051E15D10B4C0B4B188023005833BC
:1083A0001870606D002802D003F086F9656525001D
:1083B00050356068002801D003F07EF90834AC42E3
:1083C000F7D170BD7065FF1FC065FF1FF0B51700C6
:1083D000A12285B0920001934243394B06001B68ED
:1083E0000C009B18D933FF331D78FDF741FF043093
:1083F000854204DD3000FDF73BFF0430C5B2BD42CD
:1084000007D33A0000213000019B03F0DDF805B0EE
:10841000F0BD2900380002F0AFFF2300C6B2503390
:108420001E700393019B29006365380002F08CFFE6
:10843000CBB20293002B02D0039B01361E700026A4
:108440002300503303931B78B34204D8606D002897
:1084500031D10020DBE7029A2800002A04D0013B3A
:108460001000B34200D02800F700E719387002F07E
:10847000ABFF786000280ED03A78019903F08CF8B1
:10848000019A3B780136D3180E4A0193D369F6B2AC
:108490000133D361D4E7039B18706065A74205D10F
:1084A000084A1320D36A0133D362B0E7606803F04F
:1084B00003F90834F2E703F0FFF800236365C8E727
:1084C0003409FF1F3C65FF1FF7B50D0007000421AD
:1084D000686803F069F82B89040003702B891B0A74
:1084E00043702B8883702B881B0AC3702E8902254A
:1084F0000436F6B2F42E15D81B4B9F4214D10C2033
:1085000003F0E2F91135011E0CD0902303708E3B6D
:108510000371043B4380154B8460C680187803F0D8
:1085200013F800252800FEBD5C237B43104AD318B6
:108530000093583301931B78002B0FD103003200B6
:1085400038000099FFF742FF019B05001B78002BC4
:10855000E8D13800009903F097F8E3E7054A0725CA
:10856000536A01335362DDE7FEFF00003465FF1FED
:108570007065FF1F3C65FF1FF0B587B000901720A6
:108580000F0016000193FFF7F2FD1325041E19D00A
:108590000C98031E02D00199201D9847030AE3702E
:1085A000052302AAA070043090812770009866709D
:1085B00003A993800494FFF787FF051E02D02000D3
:1085C00003F07AF8280007B0F0BD0000F0B587B0DE
:1085D0001F000CAB1B780391059301210DAB060026
:1085E0001C78049200F0D6F81425002821D0200031
:1085F000FFF77EFD0135041E1BD01149059B0A784B
:1086000003700132D2B2131EC68001D101231A00B9
:108610000B7022713000049B03990097FFF7ACFFA9
:10862000051E09D1230021000648074A093303F03B
:10863000B3F9280007B0F0BD002363802370F8E78A
:108640003865FF1FC780001130750000F8B50500C0
:108650000E00064C064F2368002B02D03100280084
:1086600098470434BC42F6D1F8BDC046DC65FF1F14
:10867000F065FF1F0123064A5B42538000231371FC
:108680005362044A136053609360D3601361704770
:10869000F065FF1FDC65FF1F0200002310B50649CF
:1086A0009C000859002801D1625010BD0133052BF0
:1086B000F6D11320F9E7C046DC65FF1F034A538853
:1086C000181A43425841404210407047F065FF1F5E
:1086D000F0B585B002930AAB1F780CAB1B880090F5
:1086E00008000E0001920393FFF7E8FF0500112038
:1086F000002D1BD10E48FFF7E1FF04001520002CD0
:1087000014D006220B99A771E01D02F045FF019BD2
:1087100030002371029B29006371009B66802370E7
:10872000039B6562E381FFF791FF280005B0F0BD70
:10873000FFFF000010B5FFF7C1FF04000220002C6E
:1087400012D060880121FFF781FF606A002801D004
:1087500003F0AAF828220021200003F0ADF801233D
:1087600000205B426380207110BD000030B5074AD5
:10877000074C5588010013780020A54204D05B1AED
:1087800059424B415842104030BDC046F065FF1F72
:10879000FFFF0000084A10B501230C00904208D0EA
:1087A000FFF78CFF031E04D0037923405A1E934128
:1087B000DBB2180010BDC046FEFF0000024B187966
:1087C000431E9841C0B27047F065FF1F70B50400AA
:1087D0000D001600FFF772FF002804D10D4B9C42DC
:1087E00000D0143070BD416A03790520002907D0FC
:1087F00012221A40102A02D10520002EF2D10F2099
:10880000DB06EFD5897E0C20A942894149424942C5
:108810000840E7E7FEFF0000030010B5002800D184
:1088200010BD0348034A41889142F9D09847F7E7C1
:10883000F065FF1FFFFF0000002330B5C45CCD5C76
:108840006C40D4540133102BF8D130BD0F230022DB
:1088500010B5C45C64002243CA54C25CD209013B17
:10886000F7D210BD0200010010B52032103102F025
:10887000CBFE10BDF0B58BB0039010200593170010
:10888000049102F0D9FE0090102002F0D5FE009B6A
:1088900013240190002B05D000280CD1132400983C
:1088A00003F002F8019B002B02D0180002F0FCFF3D
:1088B00020000BB0F0BD102002F0BEFE060010201C
:1088C00002F0BAFE13240500002E00D1AEE000280D
:1088D00019D01022002102F0EFFF32002900039886
:1088E00002F092FE041E0ED133787F2B51D8300057
:1088F0000099FFF7ABFF009B1B787F2B53D80199A2
:108900000098FFF7A3FF300002F0CEFF002D02D049
:10891000280002F0C9FF002CC1D1102002F08CFE0B
:108920000600102002F088FE0290002E7CD0002865
:1089300078D03A000F3223000125121105D00F33F1
:108940003B4015B25A4253411BB26A1E1201002B22
:1089500033D0049BD2B298180099029AFFF76CFFAB
:10896000013D10220021300002F0A6FFADB2049FAD
:108970002D017D19AF4242D0002C33D0300002F0DF
:1089800093FF029B002B00D189E7180002F08CFFB7
:1089900085E729003000FFF759FF28002549009A94
:1089A000FFF74AFFA7E729000098FFF74FFF2800CD
:1089B0002049019AFFF740FFA5E70F210F400499D6
:1089C0008A18D9B28F4208D9D15C06A8195401334C
:1089D000102BF6D1029A0199C0E7791A4842414119
:1089E000C901F2E73900300006AAFFF725FF32007F
:1089F000039806A902F008FE10370400BAE7002C1D
:108A0000BCD13000029906AAFFF716FF320006A972
:108A1000039802F0F9FD082204003100059802F0E5
:108A2000BBFDABE71324A9E71324AAE7002800D075
:108A30006EE733E7D0BB0011F0B58BB00F00160026
:108A40000225009000283FD0002A3DD00B1DDBB24C
:108A50001800029302F0F0FD1135041E34D0FDF72A
:108A600047FD05003A000099201D02F0D5FEEBB24B
:108A70000393E3702B0CDBB22F0A00936370FFB2F9
:108A80002B0E2370A7700193FDF72CFD102201001F
:108A900006A802F0C1FE2100029A04AB06A8FFF767
:108AA000E9FE051E0DD1039B08223370009B04A92B
:108AB000B370019B7770F370301D02F0ADFEFDF7CF
:108AC0001DFD200002F0F0FE28000BB0F0BDF0B557
:108AD0008FB00D00149E039004920593002A03D1D9
:108AE000022420000FB0F0BD002EF9D00398FFF74C
:108AF000E5FD1424071EF4D07278337812021A436D
:108B0000B3781B041343F27812061A43036A0192E6
:108B1000934201D30133E3D1002D03D03B790124EB
:108B20009B07DED50822002106A802F0C5FE059BA2
:108B300013240433DBB21800029302F07DFD051EFE
:108B4000CFD0059A0499043002F066FE0422310069
:108B5000280002F061FE3900102210310AA802F04C
:108B60005BFE2900029A06AB0AA8FFF783FE041EEB
:108B70000FD1082206A908A802F04EFE0822311DD6
:108B800008A802F079FD012807D101990398FDF7A3
:108B9000C9FC280002F088FEA3E70124F9E70000E1
:108BA00070B51C4C05002368181E10D0002D14D180
:108BB0001A78002A0CD1981C083202F0EDFC02F061
:108BC0002BFC0135002808D123681D70012070BDE1
:108BD0000A331800082202F0DFFC2368002BF5D0CE
:108BE000122002F071FE061E0DD0C1232168037011
:108BF000457002311022023002F0CEFC23683100B1
:108C0000587802F0A1FC206802F04EFE0023236099
:108C1000DCE7C0461866FF1FF8B504002020FDF70A
:108C200055FB0D4EA700BB590500002B0DD00028A9
:108C30000BD0D878FF2809D108492A000C55F359E0
:108C400007480333611802F0A7FEF8BD290002F0BF
:108C5000F3FD0028F0D1F8E73466FF1F1C66FF1F04
:108C6000719E001170B5064D84006359002B05D02C
:108C7000D87802F019FCFF226359DA7070BDC04643
:108C80003466FF1F70B506008CB00C001500002183
:108C90003022684602F010FE31001022684602F0D1
:108CA000BBFD1D2021000322684402F0B5FD68468B
:108CB000FFF7D8FD2D21040003222800694402F0AB
:108CC000ABFD20000CB070BDF0B50700160097B0EA
:108CD00001931CAB1D7830221EAB00910AA8002125
:108CE0001C7802F0E9FD102239000AA802F094FD78
:108CF0001022002102A802F0DFFD0722310002A8A5
:108D000002F08AFD072202AB9818631E9C4101996C
:108D100002F082FD02AB9C732B005A1E934102AA03
:108D2000D3730021102206A802F0C6FD06221D9969
:108D300007A802F071FD1A2002ABC01806221F9985
:108D400002F06AFD102200990EA802F065FD1022C3
:108D500002AB0EA908781C78013A6040D2B20870C4
:108D600001330131002AF5D10AA8FFF77BFD10225B
:108D700012A904000EA802F00FFC102206AB0EA9E7
:108D800008781D78013A6840D2B208700133013189
:108D9000002AF5D10AA8FFF765FD044310222098A8
:108DA000E4B212A902F038FD200017B0F0BD70B592
:108DB0000E0014008CB00100102268461D0002F065
:108DC0002BFD3100082204A802F026FD2100082214
:108DD00006A802F021FD6846FFF744FD04001022BA
:108DE000280008A902F018FD20000CB070BDF8B5ED
:108DF00006000D0000243719AC4200D3F8BD02F084
:108E000023FC030A3B70631CDBB201379D4203D98C
:108E10000234F054E4B2EEE71C00EDE773B506004F
:108E20000C000225002819D0002917D0032101A821
:108E3000FFF7DDFF6B469A793F231A400133134356
:108E40006A463000937101A92200FFF71BFF051E3F
:108E500004D10322E01C01A902F09EFB280076BD8C
:108E600003785807DA08C00FD20080009B07104330
:108E70009B0F1843C0B2704707230B40C908C900B5
:108E80000B4303707047000070B50400FFF7EAFE63
:108E9000134DA4006359002B21D0186A002801D07B
:108EA00002F002FD2B59986E002801D002F0FCFC64
:108EB0002B59D86E002801D002F0F6FC2B59186F00
:108EC000002801D002F0F0FC2B59586F002801D087
:108ED00002F0EAFC285902F0E7FC00232B5170BD98
:108EE0003466FF1F0E4B8000C35870B50C00002B7A
:108EF0000FD09D68002D0CD02B78201D0B706B7847
:108F00004B70A97CFFF7B8FF2B7E23726B69E3607F
:108F100070BD10220021200002F0CEFCF8E7C04610
:108F20003466FF1F014B18607047C0463066FF1F54
:108F3000074A03008000825810B5002A06D0D08866
:108F4000984203D1012901D1FFF79EFF10BDC04611
:108F50003466FF1FF0B5264E95B087000B93BB59C2
:108F60000500099112200A92002B31D0D888FFF712
:108F7000A5FB04001420002C2AD0280010A9FFF71C
:108F8000B1FFBB591E781D6A002E23D00895FDF74E
:108F9000EFFA07000020FDF7F1FA0790A379E61D2C
:108FA000069310AD0CA9089800F0E2FA0EA928006B
:108FB00000F0D7FA0B9B0A990493069B0998029339
:108FC000079B0396019300970EAB0CAAFFF77CFE5C
:108FD00015B0F0BDFDF7CCFA06903000FDF7CEFAE3
:108FE000E31DA779079310AB06000893DAE7C046A4
:108FF0003466FF1F30B50C4C85002A59030085B03C
:109000000120002A0ED018006946FFF76BFF2B598C
:109010001A78D888054B002A00D1054B6A460721EB
:1090200000F0D9FB05B030BD3466FF1F6395001119
:109030007195001130B5094C8500295985B0102271
:109040006846253102F0A8FA2A591121044BD0882C
:109050006A4600F0C0FB05B030BDC0463466FF1F55
:109060000D96001130B5094C8500295985B01022A4
:109070006846353102F090FA2A591121044BD08804
:109080006A4600F0A8FB05B030BDC0463466FF1F3D
:109090004B960011F7B54D4F86001020F4590D0086
:1090A00002F0CAFAF3592062186A132200286CD021
:1090B000033A29009C6802F06FFAF3591A7801927A
:1090C000002A58D11E6A227D317B944651400122EC
:1090D000019F114201D167461740217D91433943D9
:1090E0002175377B4F40BC4660460027800701D47E
:1090F0004F081740012102208F40227D82433A43CE
:109100002275377B5740BC4660460027400701D494
:1091100097080F400420227DBF0082433A43227506
:10912000627D002794466046727B42400A4201D12C
:1091300067460F400121627D8A433A436275777B1F
:109140005740BC4660460027800701D457080F40AF
:109150000220627D7F00824317436775767B002281
:109160007E40760701D4BA080A400426617D920049
:10917000B1430A4362756A78002A08D06278002AEF
:1091800005D005220533DA7700221000FEBD042247
:109190002979114205D1A17C114202D10533033A4C
:1091A000F1E7019A21782C78002A02D10A002100E7
:1091B000140018220429E8D8042CE6D805206043BE
:1091C000034A05331218525CDDE7C0463466FF1FC0
:1091D000E0BB001110B50A001121024B00F0FBFAB0
:1091E00010BDC046A79600110B0030B587B001AD89
:1091F0002B806B4604001100981D082202F0CCF968
:109200002A000B212000024B00F0E5FA07B030BD28
:10921000CF96001110B50A001121024B00F0DBFAC5
:1092200010BDC0462397001113B50B0011006A460C
:1092300013706B4604000622581C02F0ADF96A4612
:1092400008212000014B00F0C6FA13BD439700111E
:1092500010B50A001121024B00F0BDFA10BDC04646
:10926000939700117FB505000B4BAA00D458080056
:10927000002C0FD0666F237FE28821780396266F3B
:109280000296E66E0196A46E0094FDF709FC280094
:10929000FFF7FAFD7FBDC0463466FF1F10B51721EA
:1092A000FFF7E0FF10BD000070B50A000D00064B8F
:1092B0000221040000F08FFA060029782000FFF751
:1092C000D1FF300070BDC0467396001170B586B0F6
:1092D00000236A461370836804001D78681E0A28FC
:1092E00059D801A902F068FA060633373B3F4347D5
:1092F0004B4F5300180000F042F9062312284BD0C0
:1093000000281BD16088FFF7D9F90823002813D063
:109310004279002A47D1264B1A78072312070BD52A
:10932000244B1A680723002A06D01668002E03D0A3
:10933000290001AAB04703006A4613706B461B78E8
:109340006088002B2AD1FFF767FC06B070BD1800BB
:1093500000F06CF9D4E7180000F087F9D0E71800A6
:1093600000F093F9CCE7180000F0ADF9C8E7180059
:1093700000F0C3F9C4E7180000F0F6F9C0E71800E0
:1093800000F0F6F9BCE7180000F013FAB8E718008F
:1093900000F013FAB4E707236A4613706946608841
:1093A000FFF782FFD1E70523012AC5D1024BB8E7B9
:1093B000C164FF1F2C66FF1F3066FF1FF8B52C4FDE
:1093C0008600F35904000D00002B40D0DA88824259
:1093D0003DD15A78062A33D11A78002A2ED001209E
:1093E00099681A6A097D014206D0157B054203D0AF
:1093F00007225A700120F8BD0220014204D0157BDB
:10940000054201D00922F4E70420014204D0127B76
:10941000024201D00B22ECE7164B1B68002BE9D06F
:109420005B68002BE6D020009847BB5900215B7891
:10943000122BDFD12000FFF715FFDBE70E4BECE727
:10944000112A04D1002900D032252900F2E7002D8D
:1094500008D12000FFF732F9002803D01023027949
:109460001343037121002800FDF798FAC2E7C046B4
:109470003466FF1F2C66FF1F3066FF1F70B50E4E4F
:109480008500AB590400002B13D01B78002B11D1A1
:109490000A4B1B68002B04D05B68002B01D0200016
:1094A000984773595B78122B03D100212000FFF7F6
:1094B000D9FE70BD024BECE73466FF1F3066FF1F1C
:1094C0002C66FF1F094B8000C3581020002B0CD0C6
:1094D0001A6A002A09D09B68002B06D0127A1B7EDC
:1094E000101C9A4200D9181CC0B270473466FF1F86
:1094F00070B503000D0014000220002A30D00029AE
:109500002ED013700B78081D53704B789370FFF7B3
:10951000A7FCE070012002212B7A23716B7B0340B2
:1095200063716A7B0A401343042263716E7B1640A9
:10953000334363716E7BF608F600334363712B7B14
:109540000340A371287B014000200B43A371297BBA
:109550000A401343A3712A7BD208D2001343A3719C
:1095600070BD10B50A0001000120FFF7C1FF10BD5A
:1095700010B50A0001000220FFF7BAFF10BD70B558
:1095800006000C000220002E30D000292ED0737867
:10959000201D0B70B3784B70F178FFF76DFC012242
:1095A0003579257271794B100800134093401040B3
:1095B0000343881010408000C9080343C9000B43CF
:1095C0006373B1794B10080013409340104003437C
:1095D000881002409200C9081343C9000B432120A0
:1095E0002373FCF773FE854201D2122070BD222046
:1095F000257AFCF76BFE8542F7D823781820042BD8
:10960000F4D86378012BF1D80020EFE7030010B500
:109610000220002909D0002B07D00322481C0A7021
:1096200019000D3201F0B8FF002010BD0300022226
:10963000080010B5002B06D0002904D00E32591CAA
:1096400001F0AAFF0022100010BD030010B5022097
:10965000002909D0002B07D00422481C0A701900E9
:109660000C3201F099FF002010BD10B5FFF7DEFFAE
:1096700010BD03000220002906D0002B04D00522D3
:1096800000200A701B784B70704703000220002BEB
:1096900008D0002906D05B7800200B70013B082B16
:1096A00000D918307047030010B50220002909D0F6
:1096B000002B07D00622481C0A7019000A3201F05C
:1096C0006BFF002010BD10B5FFF7B0FF10BD02000A
:1096D0000B00022010B500290ED0002A0CD0072163
:1096E0001970118859701188090A99701118082287
:1096F000D81C01F051FF002010BD03000A00022019
:1097000010B5002B0CD000290AD09978587809029E
:1097100001431180901CD91C082201F03DFF00205C
:1097200010BD030010B50220002909D0002B07D07E
:109730000822481C0A701900921801F02DFF002021
:1097400010BD02000B00022010B500290BD0002A2A
:1097500009D009211970117818185970511C062266
:1097600001F01AFF002010BD10B5FFF75FFF10BD1C
:1097700002000B00022010B5002A09D0002907D0F2
:109780005178197011180622581C01F005FF0020AD
:1097900010BD030010B50220002909D0002B07D00E
:1097A0000A22481C0A701900063201F0F5FE00205A
:1097B00010BD10B5FFF73AFF10BD02000B000220EC
:1097C00010B5002A06D0002904D018005178FFF700
:1097D00053FB002010BDF0B585B017001E006A468F
:1097E00006230500080091819380FEF7C0FC132436
:1097F000011E02900CD03800B047041E05D128008D
:1098000001A9FEF76FFA041E02D0029801F054FF7E
:109810002800FFF701FA200005B0F0BDF0B5040004
:109820008BB0019115000021102202A802F044F82B
:10983000334EA700B85900283CD0C388A34239D181
:109840000378002B36D14278062A18D10200010095
:10985000553235310C3006ABFFF7A9FA002829D173
:109860002000FFF72FFE020006A902A801F094FED7
:10987000200002A902F040F801200BB0F0BD816E7B
:10988000002917D00B8A112A28D19D420ED10198A8
:109890001231093A01F0F0FE012807D1BB5920002E
:1098A0009D6EFFF70FFE29000200DEE73221200047
:1098B000FFF7D8FC2000FEF701FF061E1BD0416A0F
:1098C000002918D00B8AAB4215D108220198123119
:1098D00001F0D2FE01280ED1716A0AE09D42E9D161
:1098E00008220198123101F0C7FE0128E2D1BB59CC
:1098F000996E8A7EB9E7200001F0A6FFBCE7C0465A
:109900003466FF1FF0B56B4D87007E5985B0337804
:1099100002900393002B00D087E0B368346A019370
:109920007078062817D101221B7D134202D0217BBB
:10993000114218D10222134202D0217B114251D18F
:109940000422134203D0237B134200D08BE0019BFF
:109950005A7DEB5991E007380428F8D801F02CFF24
:10996000032E42678300B36E002B03D11C2001F04D
:1099700063FEB066EB599C6E002C1CD010220021B7
:10998000200001F099FF0298FFF79CFD01002000E4
:10999000FFF72DFA01F058FE208220000821123036
:1099A000FFF725FA0298FFF78DFDA076EB5921000D
:1099B000D888FFF70FFC0822EB591CE0B36E002B90
:1099C00005D01A00198AF0881232FFF70DFC022226
:1099D000019B197DEB5911423DD0207B10423AD0BA
:1099E000073208E0F488FCF7DBFD01002000FFF7F8
:1099F00011FC0A22EB595A70029B9C002A59537899
:109A0000073B042B11D8D088FEF758FE00284ED013
:109A1000C3895A08D2182849029B0298CB542B5963
:109A200041180433254801F0B7FF05B0F0BDFCF73D
:109A30009FFD03000120834201D100200393EB59D5
:109A4000DE88FCF79BFD039902003000FFF7ECFB7A
:109A5000019AEB59117D042211420CD0217B114255
:109A600009D00B22C7E7F688FCF73CFD0100300067
:109A7000FFF7EEFB6BE7019A527D01210A4204D009
:109A8000607B084201D00C22B5E702210A4204D0D3
:109A9000607B084201D00E22ADE704210A4204D0C7
:109AA000627B0A4201D01022A5E71222A3E7FA2224
:109AB0005200B0E73466FF1F3866FF1F7B9E00111F
:109AC00010B5064B1A780423100018401A4200D033
:109AD0000348FFF727FA002010BDC046C164FF1FEE
:109AE0007443FF1F70B50400FFF7D4FA051E43D17D
:109AF0002000FFF77FFA234EA400A0598268937CD0
:109B0000DB0708D50321036A1B790B40012B02D127
:109B1000017F0B430377431DD97F8B1E022B0DD88A
:109B2000022900D00121C088FCF790FF042133599D
:109B30001A7F59700A431A77280070BD01290CD189
:109B400002231022437000210C3001F0B5FE305981
:109B500010213530FFF74BF9EEE70529ECD1022350
:109B6000D118437010220C3001F016FD0423325935
:109B7000117F0B431377EAE708251828DCD1053D50
:109B8000DAE7C0463466FF1FF0B58BB00591438815
:109B90007E4F9E00F45915000493002C15D1012925
:109BA00002D000200BB0F0BD101D57781678FFF7DB
:109BB00057F9EB68320002932B7A049901930090D5
:109BC0003B002000FCF70CFFEBE7E388049A93428C
:109BD00001D00820E6E72378012B00D1D4E0059BD3
:109BE000581E092800D9CFE001F0E6FD05CE0A296C
:109BF000CC506C859AB229000498FFF773FFD1E727
:109C0000200029001022453001F0C6FCB9594B78DC
:109C1000042B02D1013B4B70C3E70B000A00253334
:109C200035320C310498FFF795F90498FFF702FAE2
:109C30000522431E9841BB59C0005A70B2E720006C
:109C400029001022553001F0A7FC049B4F4C9D00C9
:109C5000295904980A0006AB55320C31FFF77AF9FE
:109C600029591022453106A801F006FD012808D126
:109C70000498FFF7F7F90590002804D106222B5924
:109C80005A7005988EE708230593FAE763780C2B42
:109C90007AD1E36E002B03D11C2001F0CDFCE066ED
:109CA000BB59D86E00286FD01022290001F074FC37
:109CB000BB590498DC6EFFF705FC0D22A076BB595A
:109CC0005A706EE7E06E00285ED063780D2B5BD192
:109CD0002B8808220382A91C123001F05DFCBB59BD
:109CE0009A68517D0222114226D0186A407B1042A8
:109CF00022D00C32E4E763780E2B45D1236F002B82
:109D000003D1162001F098FC2067BB59186F00287A
:109D100003D01022290001F03FFC0F22BB59CFE7EE
:109D200063780F2B30D1206F0622691C103001F0B0
:109D300033FCBB599A68517D0422114203D0196A41
:109D4000497B1142D5D100210498FFF78BFA28E70F
:109D5000636F002B0DD0BB59586F0028F3D0102231
:109D6000290001F019FC0122BB5952425B6F1A61B4
:109D7000E9E7142001F060FCBB5960675B6F002BC2
:109D8000E9D126E72978DFE707200BE73466FF1FD4
:109D900010B5064C207001F0DFFC06212078FDF79D
:109DA00091FF0348FEF778FC10BDC0464766FF1FD1
:109DB000318F001100200BB270B50D00834216DA0E
:109DC000264B187801F0C0FD041E0DD00378922BAD
:109DD0000ED0A02B37D0224B1878FF283AD0210084
:109DE00001F0B2FB002835D180200002684070BD30
:109DF00043780E2B0BD03E2BEDD18378052B12D060
:109E0000082BE8D181798088FFF7D8FA08E0154B54
:109E100082889A42DFD183681878591CFEF7C0FE09
:109E2000002817D1D7E7104B1B785B0712D50F4BD3
:109E30001B68002B0ED09B68002B0BD0C289811DA4
:109E400080889847ECE7FFF741FAA068002801D026
:109E500001F032FC200001F02FFBC5E74766FF1F31
:109E60006D43FF1F18200000C164FF1F3066FF1FF5
:109E700010B50078FFF712FA10BD10B50078FFF7A3
:109E8000FDFA10BD0C234343084A10B59B185A68CD
:109E9000002A03D0012901D1904710BD9B68002BF7
:109EA000FBD00029F9D19847F7E7C0466466FF1F49
:109EB00001238340094A10B5946B1C439463506B93
:109EC00098435063D46B20009843012901D12000AE
:109ED0001843D063116B0B43136310BD0080004027
:109EE000F0B500240127154B85B0DA6B144E0392B0
:109EF0001A6C0192DA64019BE3403B4217D0039D48
:109F0000E5403D400295E5B202992800FFF7BAFF0F
:109F1000316A736A002908D03900002B01D00299F8
:109F200079402800FFF7C4FF01E0002BF9D101348C
:109F30000C36172CDFD105B0F0BDC04600800040C4
:109F40004866FF1F064B01215A68C2400A4204D0EE
:109F50001B68C3401800084070471B6DF9E7C046F6
:109F6000008000400122064B8240002903D0D968BE
:109F70000A43DA607047D9689143D960FAE7C0466E
:109F80000038004030B5032444430F4BE25C1B19FA
:109F90009C785D7801232D1B0135AB40013BA3402C
:109FA000A140DB430C00122807D808499200521840
:109FB000116819402143116030BD054A11680B40FA
:109FC00023431360F8E7C04627BC001108F00040A7
:109FD00014F00040C21F70B5D4B20623092C0BD870
:109FE0000125084C9540002908D00021FFF7CAFF41
:109FF00023682B4323600023180070BD2368AB4304
:10A00000F8E7C04600380040214BF0B51B185B78DC
:10A01000022B21D1032444431E4A1F4EA35C121974
:10A020009478012215008540B76B013CE4B23D43B2
:10A03000A240B563194C122815D89B0000290CD1F9
:10A0400017495B1899680A439A600123205C154AF6
:10A05000834011680B431360F0BD11495B18996888
:10A0600091439960F1E70E4B00290DD159690A43DC
:10A070005A61225C1328E8D00123203A93400A4910
:10A08000086803430B60E7E7596991435961F0E7BA
:10A090004866FF1F27BC0011008000406CBC001107
:10A0A00000F00040A0F00040A4F00040F8B500240B
:10A0B0001B4E1C4D1C4B1B5D012B1FD1194A926975
:10A0C000E2401A420BD00122B25693402200143AC9
:10A0D000D2B2022A09D815494A6913434B610134A7
:10A0E00002360C35172CE5D1F8BD0022B2560F49C7
:10A0F0009200521891680B439360F0E7022BEED167
:10A10000E7B23800FFF71EFF01235840C1B2380004
:10A11000FFF77AFF3800FFF715FF6877DFE7C046E3
:10A12000F9BB00114866FF1F4966FF1F00F00040A1
:10A13000012202388240054B002903D059690A43A5
:10A140005A617047596991435961FAE700380040F4
:10A15000F8B50E0001210F008740114A0400D368B2
:10A16000FD43BB43D360831E8B4201D8FFF7E0FF62
:10A1700000212000FFF72EFF0A4A0B4B5168012EE9
:10A1800005D139431B1951605E700020F8BD29408C
:10A19000516002221C1962709A6915409D61F4E7B2
:10A1A00000380040008000404866FF1F012210B5C3
:10A1B0008240074B002906D019680A431A60012122
:10A1C000FFF7C6FF10BD196891431960F7E7C04655
:10A1D000008000400C2370B5002543430A4A290043
:10A1E0009B181D70094B04001B185D70FFF7B0FF32
:10A1F0000123A340064928000A681A430A6005495A
:10A200000A689A430A6070BD6466FF1F4866FF1FB4
:10A21000348000403080004070B504000E00FF28FC
:10A2200013D003250540FFF7D5FF084AA3089B007C
:10A230009B183F22ED00AA40AE40196820009143D0
:10A24000314319600121FFF78DFE70BD18380040C1
:10A25000F8B50C244443134B0500E4186368002B45
:10A2600003D1A3681220002B1AD0022201270E4B23
:10A2700000215B195A7028002770FFF769FF636897
:10A280001E1E08D0A3683E00002B04D02800FFF754
:10A2900059FE4640F6B228003100FFF709FE0020C3
:10A2A000F8BDC0466466FF1F4866FF1FF7B5C420AF
:10A2B000FF222B4B80001958002491433F3A0A4358
:10A2C0001A508022274F5202274E1A60274B1D5DDD
:10A2D000002D21D0A31E012B03D80121E0B2FFF7EE
:10A2E00027FF012D18D11F4B9B69E3402B4213D050
:10A2F000E3B218000193FFF725FE01000198FFF774
:10A3000055FFE3B2143B022B1DD801217156184AA8
:10A310008D405369AB4353613B7F002B0DD0E5B2B9
:10A320002800FFF795FF2800FFF70CFE7B7F010058
:10A33000834202D02800FFF7A5FD01340C37023616
:10A34000172CC3D1F7BD012100237156F3568D4060
:10A35000074A9B009B189A68AA439A60DCE7C046AC
:10A3600000E100E04866FF1FF9BB00114966FF1FCE
:10A3700000F0004010B501210400FFF7E9FE0123C1
:10A38000044A002011194B70A34091690B4393615B
:10A3900010BDC0464866FF1F70B50E0015000400D2
:10A3A000FFF718FF0C236343094A20009B189D60A8
:10A3B0005E60FFF74DFFF021064B074A8900051E3E
:10A3C0005A5002D02000FFF705FF280070BDC0469C
:10A3D0006466FF1F0000FF1FE19E001170B5134D62
:10A3E00007202C78002C1FD1982221005200280031
:10A3F00000F0B2FF0123C420FF222B700C4B800021
:10A400001C635C630B4B1C605C600B4B19589143E5
:10A410003F3A0A431A50802252021A600D20074A1E
:10A42000074900F0B9FF200070BDC0464866FF1F15
:10A4300000800040A0F0004000E100E0ADA200116B
:10A44000ADA00011030010B50620072B09D8054A5E
:10A45000137001F021F9D7210020034B034A890032
:10A460005A5010BD9C43FF1F0000FF1FC91BFF1F58
:10A4700070B51D0002240C2910D8094ACA40D20721
:10A480000CD5FBF72FFF041E08D1059A049928006C
:10A49000FBF744FFFCF7B2FDFFF712FB200070BD95
:10A4A0001210000030B50D7802232C009C43184296
:10A4B00001D02B431C0008252300AB43284201D0C8
:10A4C0002B00234320241D00A543204201D01C4320
:10A4D00025002A230D70184204D011781E3B0B432F
:10A4E000137030BD0028FCD10C2113788B43F7E7A3
:10A4F000F8B51D0006AB1B88140007AA0E000B2040
:10A500001778002B27D10A78022A49D14A68507857
:10A5100011780002244A08438018042840D801F02A
:10A520004BF903121D1B2300F06800F0CDFF021C45
:10A53000C0B2B84200D93A1CD2B22000F1682A80D9
:10A5400001F02AF806E00222F3681B882A802370B3
:10A550001B0A63700020F8BD0622EEE701232B8062
:10A56000F3681B782370F5E7F368002B16D00822F8
:10A570002A801A8822701A88120A62705A88A27079
:10A580005A88120AE2709A8822719A88120A6271B5
:10A59000DA88A271DB881B0AE371DBE72B80D9E73D
:10A5A00001202B80D7E7C04600D6FFFFF7B5160085
:10A5B0000A781D0008AB1F880C000123022A18D15D
:10A5C0004A685078117800022B4A08438018032803
:10A5D0000FD801F0F1F802254439E06800F074FF6B
:10A5E000C0B20723B84204D37B190193152B02DDB7
:10A5F0000D231800FEBDE0682A003100C01900F0EC
:10A60000CBFF6B4600209B88E268D0541B4B1B6835
:10A61000834203D01B68834200D098470023E8E7B9
:10A620000B23002FE5D1022DE2D1737832781B0283
:10A630001343E2681380114B1B68002BEED01B689C
:10A64000002BEBD00120E8E70B23002FD1D1062D02
:10A65000CED12A003100E06800F09EFFDEE70B2338
:10A66000002FC6D1012DC3D132787533012AC0D84D
:10A67000E3681A70D2E7C04600D6FFFF5468FF1F98
:10A6800070B50C001500072837D801F095F80414B0
:10A6900036361B36242E182015290BD8184E1622B4
:10A6A0000021300001F008F922002900300000F0FC
:10A6B00073FF002070BD18200229FBD11288114BB6
:10A6C0001A80F6E718200829F4D10A000E4829005C
:10A6D00001F02AF9EDE718200129EBD10B4B107896
:10A6E0000B49DA69FFF7DEFEE3E718200129E1D123
:10A6F000064B10780749DA6BF4E70220DAE7C04628
:10A700003C68FF1F1A44FF1F1044FF1FA043FF1F98
:10A71000C843FF1FE843FF1F030010B50020DB07FD
:10A7200004D50721024A034800F08CF810BDC0464A
:10A7300084BC0011A043FF1F054A030010680028D5
:10A7400003D082889A4201D1806870470068F6E79A
:10A750004C6AFF1F0A88030008009A4204D08A88C6
:10A7600004309A4200D0002070470000F8B5F22271
:10A7700000230D4F0D4E7968050042433370994216
:10A7800000D07B600A4C0021200001F095F80023E6
:10A790001A007C60AB4202D100203370F8BD013357
:10A7A0002280DBB2F234F5E7446BFF1F426BFF1FE0
:10A7B000506AFF1F73B56B4601900600684615008E
:10A7C0001980FCF74DFF041E11D1002D0FD07689A2
:10A7D000002E11D00C2000F02FFF00280ED0084AC8
:10A7E0000460136886808560002B02D11060200011
:10A7F00076BD1A001B68F7E70224F8E71324F6E792
:10A800004C6AFF1F012100220A4B10B549420A4C35
:10A81000198099809A719A70084B207001201980D4
:10A820005A60FFF7A3FF2078FCF778FF0448FDF794
:10A8300033FF10BD5C68FF1F4C6BFF1F446BFF1F95
:10A84000F1A80011022310B5002802D0FFF7B2FFD3
:10A850000300180010BD0000030010B50020DB0746
:10A8600004D50421024A0348FFF7A4FF10BDC046E7
:10A8700098BC00112044FF1FF0B50E2687B003934B
:10A880000CAB1F8802ABF6180500080031000292DD
:10A89000FDF768F804000120002C0FD03088FFF786
:10A8A0004BFF03000E20002B08D05E68002E05D061
:10A8B00021002800039B029A0097B04707B0F0BD23
:10A8C0000A4B10B5984207D10122002352420A8058
:10A8D0008B708A808B7110BDFFF73CFF0028FAD087
:10A8E00001235B42038000238370F4E7FFFF000035
:10A8F000F8B5050001290AD1134E00243388F22748
:10A90000AB4219D028001149FFF7DAFF06E002290F
:10A9100004D10139FDF73EFF0028EDD0F8BD3B0022
:10A9200063437268D018D35A002B09D03A00002133
:10A9300000F0C2FF0134E4B2054B1B78A342EED80D
:10A9400001235B423380DDE7446BFF1F5C68FF1F20
:10A95000426BFF1F10B5FFF7FDFE0300002083428E
:10A9600000D0987810BD0000F0B589B01C000EAB87
:10A9700080CB03901E8810AB1B78049202930B7A55
:10A980000D00DB0616D42B780593022B24D00498F7
:10A99000FFF7D2FE002812D003689C46002B0ED091
:10A9A000029B2200019329003B0064460398009615
:10A9B000A04705E00498FFF7BFFE002802D10E2053
:10A9C00009B0F0BD8368002BF9D00A222900039852
:10A9D00098470028D7D0F3E76B6858781A786B4B04
:10A9E000000210439842D2D8043B984210D2684BE0
:10A9F000984242D015D8674BC0180128C7D80B2001
:10AA0000002EDDD1EB681A7859683A80200028E0E2
:10AA1000614BC018032800D979E000F0CDFE846AAC
:10AA2000789E5E4B9842B2D10B20002EC8D10123F4
:10AA30003B80EB6831001B7823706889013080B25D
:10AA4000FCF790FF3A88031E0ED0017802328A1874
:10AA50003A80428962704289120AA270596802786B
:10AA6000E01C00F099FD06E004323A803100042237
:10AA7000601C00F021FF0020A2E70B20002E9FD1D8
:10AA8000EB6807A91E8804233B80330A3000267038
:10AA90006370FCF767FF051E28D004AB9A890E236C
:10AAA00004A95B183E49C668FCF7D0FF00280BD10B
:10AAB0002B783C486A680599FBF786FB002803D190
:10AAC000012304AA5B42D3813278022A06D171683D
:10AAD000201D00F061FD3B8802333B800E2304AA59
:10AAE0009B181B88A3701B0AE370C4E704ABDE81CC
:10AAF000F4E70B20002E00D062E7E9680398FFF727
:10AB000029FF02233B802070000A6070B3E70B200E
:10AB1000002E00D054E70222EB681B883A80237095
:10AB20001B0A6370A7E7E86800F0CEFCC2B203001E
:10AB30000720B24200D243E70DD00299DBB2711870
:10AB4000994202DB921BD3B20293029BE9681A007E
:10AB50003B8089195AE70023F6E70B20002E00D02E
:10AB60002EE70722EB683A801A7822705A786270D2
:10AB70005A88A2705A88120AE2701A792271DA8809
:10AB80006271DB881B0AA37175E7C04604290000C7
:10AB90000228000000D8FFFFFFD6FFFF03280000B7
:10ABA000FFFF0000C8BB0011F0B58DB06B46002060
:10ABB000089120229B5E83423DDAA64B187800F074
:10ABC000C3FE071E32D00378B02B2CD10079023897
:10ABD00016281FD800F0C8FB17001E001E001E001C
:10ABE00031001E0096001E001D011E0052011E00B5
:10ABF00073011E00CD011E0050021E001E001E002B
:10AC00008E021E00E302944B94491B8878880B80C7
:10AC1000FBF71AF83800FCF79BFF914B1B68002BE1
:10AC200001D038009847380000F046FC8020089B8F
:10AC30000002434018000DB0F0BDEE22002187480D
:10AC400000F03AFE0BAA3B7B7989388900923A00E2
:10AC50000D32FCF79FFD0400804B1B78002C3FD188
:10AC600046E0804B788805937F4B4100CB5A0BAE72
:10AC7000073BDBB232880293002301937B4B210018
:10AC800006930093059BFFF76FFE744D002810D1CB
:10AC9000069B3A8A1B889A420BD1380005991230DC
:10ACA00000F0EAFC002804D02B7862899B00EB18A6
:10ACB0005A80162306A81B18328820007989FCF7D1
:10ACC000C5FE2B7804009A00AA1851880029C3D029
:10ACD0000133DBB22B70002807D006A9C98A918006
:10ACE000634A12889A42BCD802E00121494291800D
:10ACF000002B04D059497888FAF7DAFF8AE73E89B1
:10AD00000A2479E000253E89574B06937B88069AF2
:10AD10005B009B5A033B9D4202DB002DF0D05BE0C1
:10AD2000162206A812183B7B798900923A0030005F
:10AD30000D32FCF72FFD0590002858D04689017A86
:10AD40007888FCF7F1FC041E44D1464B78880793C1
:10AD5000069B4100C95A454B0439C9B206AAD28A9A
:10AD600006930291019400930599079BFFF7FCFD60
:10AD7000041E2FD1069B39491A88931C002D26D119
:10AD80004B807988384B4900CB5A5119033B8B4291
:10AD900020DD059B31485B8941190B71A91C0135E8
:10ADA000C9B2EDB2059145191B0A2B71059B2D49BE
:10ADB0000433181800F0F0FB2C4B059A1B88D318AD
:10ADC000DDB22C4B9E4205D00136B6B29CE74988D5
:10ADD0009942D6D0002D0CD0204C2800618800F07C
:10ADE000FBFB207021007888FAF772FF12E7059CC0
:10ADF000F0E7002C00D183E77B78142B00D109E722
:10AE000016493B794E800B700C717888FAF712FF67
:10AE100000E7162406ABE41821003889FCF7A2FDF0
:10AE2000011E00D1B7E1788822880F4C45002C5BC9
:10AE30000A4D013CE4B2029400240F4B01940095AA
:10AE4000FFF792FD041E00D014E129007888FAF77C
:10AE50004FFFDFE64C6BFF1F0C43FF1F6468FF1FB3
:10AE60005868FF1F5869FF1F9464FF1F486AFF1F3F
:10AE70000A43FF1FFFFF00006668FF1F162406AB92
:10AE8000E41821003889FCF76DFD011E00D182E134
:10AE900078882288AE4C45002C5BAE4D013CE4B274
:10AEA00002947C89AC4B01940095FFF75DFD041E74
:10AEB00000D0DFE029007888FAF724FFAAE6002511
:10AEC000A44B1D803B00F6331B78A24A788807927A
:10AED000AB4208D99E4B12880693069943005B5AF1
:10AEE000013B9A4203DB0799FAF716FF92E6162414
:10AEF0006B00FB18059306ABE418059B210018892D
:10AF0000FCF730FD011E03D1059B01241E8973E768
:10AF10007888924B2288069C099343001B5B904ED5
:10AF2000013BDBB20293002300960193099BFFF7DC
:10AF30001BFD041E02D0059B1E895DE77B88069AD7
:10AF40005B009B5A079A108832881218934202DCE1
:10AF50001B1A013B33807F4C02303288099900195B
:10AF600000F01AFB2388328801359B182380EDB24C
:10AF7000A8E70BAA3B7B7989388900923A000D3209
:10AF8000FCF708FC00250590059B002B04D10A2442
:10AF9000002D00D16EE060E0059B7888197AFCF7FF
:10AFA000C3FB0100041E63D1694C6C4B7888069486
:10AFB0000993069B4400E45A694B063CE4B20BAE8D
:10AFC000328807930294019100930599099BFFF73A
:10AFD000CBFC041E4CD1079B5E491B881A1D002D1B
:10AFE00030D14A80059B5B4C5A8963191A716B1CDE
:10AFF0009BB2E318120A1A71162306A832881B188E
:10B0000079890598FCF722FDFF21AA1C2E1D033526
:10B010000B00059092B2B6B2ADB2002803D006ABD9
:10B02000DB8AD9B21B0AA218651911712B714C4D1C
:10B03000301D2A884949201800F0AEFA2B88F618EE
:10B04000B5B2A1E74988914207D17A8806995200A2
:10B05000525AEB18053A9A42C4DC3E4C28006188EB
:10B0600000F08AF9207021007888FAF75FFED1E5B8
:10B07000002DF2D13E89BFE6162606ABF618310048
:10B080003889FCF76FFC3D000400FA3500282DD00C
:10B09000037A9B060CD400227B8939897888009238
:10B0A0003A000C32FFF7E8FB041E10D03E8915E091
:10B0B0003088FFF741FB00281AD08368002B17D097
:10B0C0002100122278889847041EE4D0EEE72B78FE
:10B0D000002B02D17888FAF739FE00262B78002B56
:10B0E00000D097E5002C00D194E585E60124DDE74A
:10B0F0000E24DBE7162506ABED1829003889FCF78E
:10B1000031FC041E47D0037A9B0611D4154A7B8874
:10B110001188994203D01448814207D11380134B00
:10B12000F2261D780023D9B2A94221D30924A1E730
:10B130002888FFF701FB00282FD08368002B2CD034
:10B140002100122278889847041EDFD092E7C0467B
:10B150009464FF1F6468FF1F6668FF1F5869FF1F24
:10B16000486AFF1F446BFF1FFFFF0000426BFF1F79
:10B1700031005943546801336018615A0029D2D113
:10B180003C0008342100F22200F006FA2100788801
:10B19000FAF7E4FD3EE501246CE70E246AE71D4B57
:10B1A0001A887B889A4231D07888FAF7E1FD31E538
:10B1B000F223059851684343CD18C95A00291FD07E
:10B1C0003B7A012B0BD16C88AB887888AA1D009440
:10B1D000FFF752FB041E02D000233B722E88F2229E
:10B1E0000021280000F068FB00232B80059B013321
:10B1F000DBB20593084B05991B78064A8B42D7D8DA
:10B2000001235B421380002CCED0F5E500263400EC
:10B210000596EFE7446BFF1F426BFF1F70B50400FC
:10B220000E001500FFF796FA031E08D131000548FD
:10B23000FFF790FA03001120002B02D01C800020A1
:10B240009D7070BDFFFF0000F8B50B4F06003B7806
:10B250000D001400FF2B0ED00A2000F035FB011E5C
:10B2600009D0B1230380002346800371C580048187
:10B27000387800F069F9F8BD6144FF1FF7B50F0099
:10B2800008A90600088809A90B240988002821D1EB
:10B290000234022B1ED1557813782D021D432B004A
:10B2A0008B4301937334002B14D1FB6830001900D9
:10B2B0000093FFF74FFB019C85420BD02A00300022
:10B2C0000099FFF7ABFF041E04D12A0030007989F2
:10B2D000FFF7BAFF2000FEBDF0B50E7885B00390F1
:10B2E0000AA805880120022E0DD14C6827786478C1
:10B2F00024023C43054FBC4205D10398DBB20196C2
:10B300000095FFF7BBFF05B0F0BDC0460229000065
:10B31000034B10B51B68002B00D09847FEE7C046D2
:10B32000506BFF1F07B501A8FFF7F2FF044A05485D
:10B330000021121A00F010F8F8F79EFAFEE7C04656
:10B34000546BFF1F6444FF1F01B40248844601BCD4
:10B35000604700BF090E000001B40248844601BCEA
:10B36000604700BFB70E000001B40248844601BC2C
:10B37000604700BF853BFF1F01B40248844601BC03
:10B38000604700BF090E000001B40248844601BCBA
:10B39000604700BFC539FF1F01B40248844601BCA5
:10B3A000604700BF4931FF1F01B40248844601BC19
:10B3B000604700BF9137FF1F01B40248844601BCBB
:10B3C000604700BF4D39FF1F01B40248844601BCED
:10B3D000604700BF017F000001B40248844601BC01
:10B3E000604700BF8B52010001B40248844601BC93
:10B3F000604700BF456B010001B40248844601BCB0
:10B40000604700BFB352010001B40248844601BC4A
:10B41000604700BFA930FF1F01B40248844601BC49
:10B42000604700BFD91B000001B40248844601BC3C
:10B43000604700BF5D3BFF1F01B40248844601BC6A
:10B44000604700BF5934FF1F01B40248844601BC65
:10B45000604700BFF30E000001B40248844601BCFF
:10B46000604700BF0D52010001B40248844601BC90
:10B47000604700BFE932FF1F01B40248844601BCA7
:10B48000604700BFC9A9000001B40248844601BC5E
:10B49000604700BFC521000001B40248844601BCDA
:10B4A000604700BF055E000001B40248844601BC4D
:10B4B000604700BF1147010001B40248844601BC47
:10B4C000604700BF434D010001B40248844601BCFF
:10B4D000604700BFDD52010001B40248844601BC50
:10B4E000604700BF4550000001B40248844601BCDB
:10B4F000604700BFDD66010001B40248844601BC1C
:10B50000604700BF056A000001B40248844601BCE0
:10B51000604700BF75A9000001B40248844601BC21
:10B52000604700BF691F000001B40248844601BCA7
:10B53000604700BF413BFF1F01B40248844601BC85
:10B54000604700BF8552010001B40248844601BC37
:10B55000604700BF594F010001B40248844601BC56
:10B56000604700BF3D18000001B40248844601BC9A
:10B57000604700BF9136FF1F01B40248844601BCFA
:10B58000604700BF2146010001B40248844601BC67
:10B59000604700BF9D36FF1F01B40248844601BCCE
:10B5A000604700BFE94C010001B40248844601BC79
:10B5B000604700BF5549010001B40248844601BC00
:10B5C000604700BF5522000001B40248844601BC18
:10B5D000604700BF0519FF1F01B40248844601BC43
:10B5E000604700BF350E000001B40248844601BC2C
:10B5F000604700BF5D17000001B40248844601BCEB
:10B60000604700BFC136FF1F01B40248844601BC39
:10B61000604700BFE548000001B40248844601BC11
:10B62000604700BF2526000001B40248844601BCE3
:10B63000604700BF8539FF1F01B40248844601BC42
:10B64000604700BF3D4B010001B40248844601BC85
:10B65000604700BF2951010001B40248844601BC83
:10B66000604700BF5952010001B40248844601BC42
:10B67000604700BF713AFF1F01B40248844601BC15
:10B68000604700BFCD4C010001B40248844601BCB4
:10B69000604700BF3119FF1F01B40248844601BC56
:10B6A000604700BFC91BFF1F01B40248844601BCAC
:10B6B000604700BFC56D010001B40248844601BC6B
:10B6C000604700BFD949010001B40248844601BC6B
:10B6D000604700BF7918000001B40248844601BCED
:10B6E000604700BFB54C010001B40248844601BC6C
:10B6F000604700BFC94A010001B40248844601BC4A
:10B70000604700BFF919FF1F01B40248844601BC1D
:10B71000604700BF851F000001B40248844601BC99
:10B72000604700BFA54F010001B40248844601BC38
:10B73000604700BFC130FF1F01B40248844601BC0E
:10B74000604700BF0124000001B40248844601BCE8
:10B75000604700BFE928000001B40248844601BCEC
:10B76000604700BFC926000001B40248844601BCFE
:10B77000604700BF291C000001B40248844601BC98
:10B78000604700BF4538FF1F01B40248844601BC32
:10B79000604700BF6571010001B40248844601BCE6
:10B7A000604700BFED3AFF1F01B40248844601BC68
:10B7B000604700BFC51D000001B40248844601BCBB
:10B7C000604700BF713BFF1F01B40248844601BCC3
:10B7D000604700BF2124000001B40248844601BC38
:10B7E000604700BF4D1F000001B40248844601BC01
:10B7F000604700BF3555000001B40248844601BCD3
:10B80000604700BF6DBC000001B40248844601BC23
:10B81000604700BF9DA9000001B40248844601BCF6
:10B82000604700BF4551010001B40248844601BC95
:10B83000604700BF5125000001B40248844601BCA6
:10B84000604700BF5147010001B40248844601BC73
:10B85000604700BF091B000001B40248844601BCD8
:10B86000604700BF156B010001B40248844601BC6B
:10B87000604700BF193BFF1F01B40248844601BC6A
:10B88000604700BFF94C010001B40248844601BC86
:10B89000604700BF8D12000001B40248844601BC1D
:10B8A000604700BFE117000001B40248844601BCB4
:10B8B000604700BF014C010001B40248844601BC4E
:10B8C000604700BF154D010001B40248844601BC29
:10B8D000604700BF1D4D010001B40248844601BC11
:10B8E000604700BF2933FF1F01B40248844601BCF2
:10B8F000604700BF692EFF1F01B40248844601BCA7
:10B90000604700BF311B000001B40248844601BCFF
:10B91000604700BF1D4B010001B40248844601BCD2
:10B92000604700BFB14E000001B40248844601BC2C
:10B93000604700BF810E000001B40248844601BC8C
:10B94000604700BF053AFF1F01B40248844601BCAE
:10B95000604700BFF54E010001B40248844601BCB7
:10B96000604700BFADAE000001B40248844601BC90
:10B97000604700BFEDA5000001B40248844601BC49
:10B98000604700BFED4A010001B40248844601BC93
:10B99000604700BF3939FF1F01B40248844601BC2B
:08B9A000604700BFA946010049
:10B9A8000003010302000303040205020602070064
:10B9B800080309030A030B030C000D000E030F0311
:10B9C800100311001303140315031603393C001167
:10B9D8006D3C00110000000002000000EAB90011EF
:10B9E800192A0F180A000000F1590000FD24000070
:10B9F80041460100A17D0011B59D00110972001199
:10BA0800A57B0011B5530011A9AB0011115000110D
:10BA1800493E0011793F0011000000001616000091
:10BA28000200000034BA0011F4FFF3FFD2FC00005A
:10BA3800B940001100000000000000005475796151
:10BA48000042322E30003030313300676974687537
:10BA5800622E636F6D2F70767678005448423200FC
:10BA6800020000007CBA0011292A282A272A262A3F
:10BA7800252A242A0A180000E204000071020000A6
:10BA880078EC00000500000074400000102700005A
:10BA980060F000000400000006640000204E000072
:10BAA80000000000060000005C44000010270000B1
:10BAB8006CEE000007000000050000001F501D107C
:10BAC800023CB400000113002000000081020000C5
:10BAD80030313233343536373839414243444546BC
:10BAE80000000000B95700110D58001100000000B7
:10BAF8000200000004BB00116F2A6E2A1A18000009
:10BB080001A00000000000006410B71DC8206E3BB3
:10BB1800AC30D9269041DC76F4516B6B5861B24D4C
:10BB28003C7105502083B8ED44930FF0E8A3D6D6B6
:10BB38008CB361CBB0C2649BD4D2D38678E20AA01E
:10BB48001CF2BDBDFB349B5F80000080001000002C
:10BB5800000000000B5E0011957400112F5E0011AB
:10BB68009D780011B35E001173780011295F0011F0
:10BB7800497800117B5F0011117A0011E35F001111
:10BB8800117A001115600011CB790011295F00119D
:10BB980001780011A15F0011A979001100000000CF
:10BBA8000000000087600011A9790011E960001108
:10BBB800AD740011052A042A012A002A0229032843
:10BBC80001280028011800180000000000000000EB
:10BBD80000000000000000870101020102010102CB
:10BBE800010203030401030101010101030302012E
:10BBF80003000D000E0010001100130014010701CE
:10BC080008010A010B011C011D02040205020702BA
:10BC1800080219021A021C021D030103020317007D
:10BC28000201000504000807000B0A001716001D92
:10BC38001C010201010504010E0D0111100114136C
:10BC4800011716011A19020201020B0A020E0D024F
:10BC58001110021413021716030504030807030B37
:10BC68000A030E0D0001020307090A0B0E0F10113B
:10BC780012141718191A1B1F20212200F1A40011F1
:10BC8800ADA500110000000002000000CEBB0011AD
:10BC980000000000D9B200110000000002000000FE
:04BCA800CCBB001100
:020000041FFFDC
:1000000000000000B13D0011F0B90011ECB9001181
:100010009461FF1F000000000000000000000000CD
:1000200000000000000000000000000000000000D0
:1000300000000000000000000000000000000000C0
:1000400000000000000000000000000000000000B0
:1000500000000000000000000000000000000000A0
:100060000000000000000000000000000000000090
:100070000000000000000000000000000000000080
:100080000000000000000000000000000000000070
:100090000000000000000000000000000000000060
:1000A0000000000000000000000000000000000050
:1000B0000000000000000000000000000000000040
:1000C0000000000000000000000000000000000030
:1000D0000000000000000000000000000000000020
:1000E0000000000000000000000000000000000010
:1000F0000000000000000000000000000000000000
:1001000000000000000000000000000000000000EF
:1001100000000000000000000000000000000000DF
:1001200000000000000000000000000000000000CF
:1001300000000000000000000000000000000000BF
:1001400000000000000000000000000000000000AF
:10015000000000000000000000000000000000009F
:10016000000000000000000000000000000000008F
:10017000000000000000000000000000000000007F
:10018000000000000000000000000000000000006F
:100190004D33FF1F9531FF1FC166010000000000B5
:1001A000000000000000000000000000000000004F
:1001B000000000000000000000000000000000003F
:1001C000000000000000000000000000000000002F
:1001D000000000000000000000000000000000001F
:1001E000000000000000000000000000000000000F
:1001F00000000000000000000000000000000000FF
:1002000000000000000000000000000000000000EE
:1002100000000000000000000000000000000000DE
:1002200000000000000000000000000000000000CE
:1002300000000000000000000000000000000000BE
:1002400000000000000000000000000000000000AE
:10025000000000000000000000000000000000009E
:10026000000000000000000000000000000000008E
:10027000000000000000000000000000000000007E
:10028000000000000000000000000000000000006E
:10029000000000000000000000000000000000005E
:1002A000000000000000000000000000000000004E
:1002B000000000000000000000000000000000003E
:1002C000000000000000000000000000000000002E
:1002D000000000000000000000000000000000001E
:1002E000000000000000000000000000000000000E
:1002F00000000000000000000000000000000000FE
:1003000000000000000000000000000000000000ED
:1003100000000000000000000000000000000000DD
:1003200000000000000000000000000000000000CD
:1003300000000000000000000000000000000000BD
:1003400000000000000000000000000000000000AD
:10035000000000000000000000000000000000009D
:10036000000000000000000000000000000000008D
:1003700025B3001100000000000000000000000094
:10038000000000000000000000000000000000006D
:10039000000000000000000000000000000000005D
:1003A000000000000000000000000000491BFF1FCB
:1003B000000000000000000000000000000000003D
:1003C000000000000000000000000000000000002D
:1003D000000000000000000000000000000000001D
:1003E000000000000000000000000000000000000D
:1003F00000000000000000000000000000000000FD
:08183800606FFF1F4118FF1F44
:10184000024981F3088802F0BFFB0000606FFF1FB0
:1018500070B500241E491F4A1F484C6308CA1B0567
:101860001B0DE4188242F9D11C4B80228B630021AE
:1018700009201B4B920519621A4B1B4DDA671B4B53
:10188000DA688243DA609A68194802409A60112047
:10189000296002F0B7F8112002F094F880226B6CF6
:1018A000112093436B64EE23DB006343114A1B0C4E
:1018B00013840122104B9A7201F022FC0F4B1B780B
:1018C000002B04D10E4B1021187802F015FB70BDCF
:1018D000000005408805054000060540FF010000A6
:1018E00000F0004004E100E0003800403CF000401F
:1018F000FFDFFFFF6461FF1F1862FF1F4664FF1FC9
:101900004462FF1F10B502F057FA072804D01228CE
:1019100008D0022808D010BD044A0420136B0133FC
:101920001363F8E70220F6E71420F4E73C65FF1F95
:10193000F8B507000C0026002500503630785135E8
:10194000002804D10300287058342370F8BD29788A
:10195000CA00481E8141A3183800A25C5B68C9B266
:10196000FFF7D0FF00280DD12B78DA00A218013341
:1019700050602B703378044A013B3370136A013393
:101980001362D8E70123DFE73C65FF1F5C23434375
:10199000074910B5C9180B0058331B78012B05D126
:1019A000FFF7C6FF034A936A0133936210BDC04636
:1019B0007065FF1F3C65FF1F10B502F03DFA064A37
:1019C0000121130010CB4942D967044B136002F088
:1019D0004BFB200010BDC04600E100E010001000ED
:1019E00010B5040002F028FA024B1C6002F03CFB28
:1019F00010BDC04600E100E010B5040002F01CFA82
:101A00004021094A200013688B43136000F0F6FA66
:101A100001F07EFC0022054B01201A60044B0432C9
:101A20001A6002F0A9F9FEE71CF00040C4F0004083
:101A3000C0F00040431E5A425341A022F0B5D201EB
:101A40005B421340154D164A40019B182A18127E1E
:101A50008BB00191002A1BD01A000832D46F0022EB
:101A6000E6B206AFE4B294420EDC2818C369002B3C
:101A700008D0019902AA117106AA049202AA16734B
:101A800003A898470BB0F0BD1978B9540132EAE7C2
:101A90001A7D1A7806AB01261A70E6E7FC67FF1F6D
:101AA00000400040F0B5254B04004001C25C85B009
:101AB000002A2BD01A18117E002927D0917E0029E8
:101AC00024D01179022921D11689D788D168F51B34
:101AD000ADB22A1C102D00D9102292B2BE4217D1ED
:101AE0001818012303710023C269C38003819A423D
:101AF00006D06846032103730171029301A8904741
:101B00000820002C00D0192001F0FAFA05B0F0BD31
:101B1000013C65426C41A0256442ED012C40084D1A
:101B20001B186419074D0633013A92B2AA42EDD050
:101B30001888461C1E80085C2070F5E7FC67FF1FB4
:101B400000400040FFFF00000F220E4B10B59868C8
:101B5000104002380A280BD802F00AF80D0A0B0AC6
:101B60000A110A0A0A0A060002210020FFF762FF92
:101B700010BD0121F9E70020FFF794FFF8E7DB6FC4
:101B8000F6E7C046004000400F220E4B10B59868A3
:101B9000104002380A280BD801F0EAFF0E0A0B0A9F
:101BA0000A120A0A0A0A060002210120FFF742FF70
:101BB00010BD01210800F9E70120FFF773FFF7E7E7
:101BC000DB6FF5E70090004013B5334C2378072B0B
:101BD0003DD8324B1A78324B002A39D1802219680D
:101BE00052020A431A60252001F0CCFE20232D4A20
:101BF00011680B43802113606B460422C9050868F5
:101C00000733104228D080210422C905C868104239
:101C10002ED080212020C905CA688243CA601422C0
:101C20001A701A78002A2FD18021C905C86820327D
:101C30000243CA6014221A701A78002A28D11A4B5B
:101C40001A7D22785A601D221A705932DA6013BD4B
:101C50001A6816490A40C5E7086802430A60142258
:101C60001A701A78002ACED01A78013AD2B2F7E761
:101C7000C8680243CA6014221A7019784A1ED2B288
:101C80001A700029F9D1C4E71A78013AD2B2C7E72D
:101C90001A78013AD2B2CEE79C43FF1F6444FF1F7B
:101CA0003CF000409443FF1F00200040FFFFFEFF78
:101CB000564B70B51B68012B03D1554A936D013308
:101CC000936501F0E9FF534B534A1860534B544C52
:101CD0001A600123534A1360534A13602378002B80
:101CE00006D006225149524801F066FF00232370B6
:101CF000504A514B10681B78C1B2002B0ED14F4C8B
:101D0000C0B223785BB2002B4FDB237824785BB220
:101D100064B21B0424021B191B1813600B1C5029EE
:101D20004ED95023464A47491078DBB2FF22022899
:101D30004BD10868444C454D267890432A7896420A
:101D400054D9227824782E78023B5D10A31B6B4374
:101D50005201D31A10335B111843086002F0ECF8FB
:101D6000031F012B45D83A4B1B78002B06D0394B6B
:101D70001B78002B02D0002001F09EFFA122364BE1
:101D800092009978354B4A431B689B188322920036
:101D90009B181B78033B012B03D8AF20400002F0B7
:101DA00013F801222E4BDA8270BD237824785BB2BF
:101DB00064B2FF33FF341B0424021B190138ABE764
:101DC000CAB2022AAED20223ACE70868254C264DDF
:101DD000267890432A78964208D9227824782D785C
:101DE000023B5B10641B63435201B2E72378DBB212
:101DF000B2E70228D5D11D4B1B78013B022B03D93A
:101E00001B4B1B78022BCCD16C20C8E79809FF1F15
:101E1000FC0FFF1F8864FF1FFF3F000014100340EA
:101E20008C64FF1F0C10034000100340D50BFF1FF4
:101E30007211FF1FB40003408C09FF1F680AFF1FC7
:101E4000490AFF1F94000340460AFF1F470AFF1F6D
:101E5000F908FF1F2209FF1F300DFF1F3409FF1F64
:101E6000BC0BFF1F440AFF1F450AFF1F1C09FF1F71
:101E70002309FF1F10B502F09FF80022014B1A80C2
:101E800010BDC0468464FF1F10B502F03DF8A121CB
:101E9000054A89009478054A61431268044B521838
:101EA000528C1A8010BDC046300DFF1F3409FF1F31
:101EB0008464FF1F10B50D4B0D4A9978A1239B0038
:101EC0004B431268D218531DD97F0A4B1B88994285
:101ED00009D2441C07D0C82805D0D2695B1A5A43DE
:101EE000054B5343C01802F057F810BD300DFF1FCB
:101EF0003409FF1F8464FF1F7102000070B5244D78
:101F00002B68002B28D001F04FFF2B68D8402B689E
:101F10000400002B27D001F0C7FE2B68D8401D4BD2
:101F20001D4A9978A1239B004B431268D118D25CBB
:101F300091239B00002A20D0CA580132CA50174B67
:101F400017491B680868834214D3D23B181A012A28
:101F50001AD0144B186070BD01F026FF124B19689F
:101F600002F052F8D3E701F09FFE0F4B196802F020
:101F70004BF8D4E70D495B18E8E7CA500C4B1B68D7
:101F8000DB68E418201AE4E7F530FF30E1E7C046EB
:101F90001C08FF1F300DFF1F3409FF1F9C09FF1F86
:101FA0008864FF1FA009FF1F1808FF1F2DFF3F00B7
:101FB0009064FF1F70B504000D00282916D103009E
:101FC000A433C2881B889B1A0B4A9BB293420DD93B
:101FD00006006A3605223100653001F085FF0028D1
:101FE00004D13100200001F03FFF70BD2900200026
:101FF00001F0F2FFF9E7C046FE7F0000F8B50500EA
:10200000012001F0B1FF134CA36AA26A9342FBD1F5
:10201000114E336001F068FE10490300086010485B
:10202000426894460F4A17680022BC4501D24268B4
:10203000BA1A0D4802603268AD18A422E562606ADF
:10204000520302436262094A1278002A01D00F3B10
:102050000B60F8BD00F00040340AFF1FE408FF1FCA
:1020600028100040180AFF1F1C0AFF1F1C09FF1F31
:1020700070B580241025E405A3682B43A36001F00C
:10208000B3FDA368AB43A36070BD0000F7B51600B5
:1020900080221C001023D2050191916805000B439A
:1020A000936000225A4BD7301A6001F0A5FE9D23A1
:1020B0002A002F009B00EB58CA3201210092FC3706
:1020C000002B01D00021009A386801F0C5FE2900DC
:1020D000009BCB311A784F4BD3351A604B780A7876
:1020E0001B0213438A7812041A43CB781B0613434E
:1020F000494A1BBA13604B790A791B0213438A7948
:1021000012041A43CB7931001B061343434A1BBA0E
:1021100013606B782A781B021343AA7812041A43BF
:10212000EB781B0613433E4A1BBA1360019A330235
:1021300013433C4A13603C4B22001B1B9C46032963
:102140003DDCB3089A0013005142B21A032A46D16B
:10215000354AE018511A827840781204000202438E
:10216000E05C043302430A600022FF2B4BDDF022C7
:102170002E4B12011A600F222D4B1A602D4A136844
:10218000002BFCD00023224A27491360091B321D73
:102190000B191B68043A180A23706070180C1B0E88
:1021A000A070E3700434002AF2DC802210213B6826
:1021B000D20501333B6093688B439360F7BD634660
:1021C000D578981893782D061B042B43157804397D
:1021D0002B43557804322D022B430360AFE7022ACC
:1021E0000AD1114AE05C511AE218527812020243F5
:1021F0000A6004339BB2B7E7012AB5D10A4A521AE2
:10220000E15C1160F5E7084959180A600433ACE74E
:10221000000004403C000440380004403400044006
:10222000300004400C00044000010440040004405D
:102230001000044014000440F7B5150080221C0073
:102240001023D2050091916807000B43936000238F
:10225000654AD730136001F0CFFD9D233E009B00FF
:10226000F9583B00CA363200FC33002900D07FE029
:10227000586801F0F1FD390032785C4BCB311A60BF
:102280004B780A781B0213438A78AC4612041A432F
:10229000CB78281D1B061343554A1BBA13604B7994
:1022A0000A791B0213438A7912041A43CB791B065D
:1022B0001343504A1BBA13604B7A0A7A1B0213432A
:1022C0008A7A12041A43CB7A21001B0613434A4A26
:1022D0001BBA1360009A2B021343484A1360220072
:1022E000474B1B1B0093009BCE785B1801938B78A8
:1022F00036061B0433430E78043833434E780431DA
:1023000036023343019E33600328ECDC0321A80826
:10231000431C9B002940800003292BD13849E51834
:102320005E18A9786D78E35C09042D0229431943EE
:102330003160030008330021FF2B2DDD314B324982
:1023400019600F21314B1960012327490B60304B75
:1023500019680029FCD006211B680B40042B20D0F3
:1023600080220020D20593680A318B439360FEBD22
:1023700001217DE7022908D121495D18E11849783A
:10238000E35C090219432960D3E70129D3D11C4931
:102390005918E35C0B60CCE7194818180160043346
:1023A000CAE7002310490B606346002B0CDC3B009E
:1023B000FC335A68102101325A608022D20593689A
:1023C00001208B439360D2E7009B9B181B68190A7E
:1023D00013705170190C1B0ED37004235B42917063
:1023E0009C440432E0E7C046000004403C00044046
:1023F0003800044034000440300004400C00044025
:102400000001044004000440080F000010000440D4
:102410001400044070B5061E19D002225A4B9B7955
:102420009343012B13D1594B1A78FF2A0FD15A78B5
:10243000FF2A0CD19A78FF2A09D1DA78FF2A06D12F
:102440001A79FF2A03D15B79FF2B00D199E0504B19
:102450000C201A78012A08D000224E4D1A702978D3
:102460000B00093B042B01D8212070BD4B1F012B11
:10247000FAD9454CA37B042B00D982E0A279032A28
:1024800000D97EE09A1ED2B2012A02D860881F28A5
:1024900077D9002E56D0012E73D1A0880128E3D021
:1024A000002907D1581E032803D801F061FB121739
:1024B00015122E702978481E032811D80025364B96
:1024C0001D602823237501F0DFFBA84227D0A580DB
:1024D000CAE702212970EDE70421FBE70321F9E7B0
:1024E00007390129C0D82D490968C96A8906BBD5B1
:1024F0002B4908780028B7D1012A01D9002BB3D184
:1025000002230B708021274D2633890128782375FB
:1025100001F002FD80212878890101F0EDFC012302
:10252000A380214B1B78002B0AD0FA2280211F4B5D
:1025300092001B8809025A431A4B187801F07CFB61
:10254000002092E701F078FC2B78A680073B012B56
:1025500003D917482E7001F0CFFB114B114C1A789C
:10256000002A06D080210022207889011A7001F00B
:10257000D3FC01F079FD80212078090201F0CCFC28
:10258000DEE7122071E7C046A60BFF1F6B09FF1F95
:102590001A09FF1F1C09FF1F4809FF1F9064FF1F36
:1025A0002309FF1F1B09FF1F2109FF1F2C09FF1F04
:1025B0000010004010B5002901D001F07DFC10BDD5
:1025C000F7B5604B01919978A1239B004B435E4A7C
:1025D000060014681022E418D6235B00E058362366
:1025E000FF33E35C00279343222B41D1574B0F3A33
:1025F0001A600760012501F0FFFC019B1880E823A9
:102600005B00E35C002B01D0B34258DD0023504F48
:10261000FB70AD33FF33E3581A68002A03D09B8860
:10262000DB439B071DD03823FF33E35C002B18D01E
:102630009B235B00E35C002B13D1D133FF33E35CBE
:10264000B3420EDAA4235B00E15AE018090A023112
:1026500001F0E2FB23000122FE33013E01351A871F
:10266000FA70E8235B00E35C002B2AD0A8B2FEBD21
:1026700003683D00002BBED081880430090A023176
:1026800001F0CAFBD6235B00E3581F60B2E72300CA
:10269000B133BA00FF339858013781880430090AF2
:1026A000023101F0B9FBE8235B00E35CBB42EEDCE6
:1026B000E822F61AED1800235200A354A6E70027DB
:1026C000F1E7200001F0C8FC00281FD0002E1DDD1E
:1026D0007319882647190193B600200001F02CFBDE
:1026E0005A30800020184068013581880430090A7A
:1026F000023101F091FB200001F04EFAA3590133A1
:10270000A351BD4202D0019B9D42E6D1114BE35C37
:10271000002BABD095239B00E35C002BA6D00E4B87
:10272000E15A0029A2D00D4AA35C994202D9013393
:10273000A3549BE700231A212000A35401F07CFC42
:1027400094E7C046300DFF1F3409FF1F00140340FB
:10275000E010FF1F5A020000720200005E0200003B
:102760000D4970B54A6E0D4CD2038B69D20BA24253
:1027700006D80B4D0224AA4204D901F045FA70BDD7
:1027800002246442E21815007E2425402242F4D03F
:10279000A3432B438B61F0E700F000400A200000C8
:1027A000FC1C0000F8B51D4B1D4F1A78002A10D1F3
:1027B000BA7B002A02D101321A7003E0032AFAD050
:1027C000022AF8D001F060FA00220120154B1A709D
:1027D000F8BD154B154D1C68154B9E7801232B70C9
:1027E0002878C0B200F09EFBBB7B002B0BD101F020
:1027F0000BFBA1239B007343E41883239B00E41885
:1028000023782B70E4E7032B02D101F065FBF0E79E
:102810000020022BDCD101F0D7F9EAE71C09FF1FE9
:10282000A60BFF1F2309FF1F3409FF1F490AFF1FC3
:10283000300DFF1FF0B587B00EAD2F780FAD2D789E
:102840000593AC46634614000E4D0CAA12782E7800
:1028500003930D9B009201932200059B029701F0C8
:102860007BFB2E70012C01D0042C08D1802206495C
:102870008B889343054A1278D20113438B8007B0AB
:10288000F0BDC0461C09FF1F6C11FF1F7809FF1F18
:102890000B001B3B70B504003020E02B0DD813005B
:1028A000E025493BFF3B9BB2ED00AB4205D8034B13
:1028B000200019825A8201F047FB70BD8410FF1F6F
:1028C00010B501F0E9F9054B00205B68052B04D930
:1028D000034A5268D20200D4980810BD001000408C
:1028E000FCE100E070B501F0A7FA0D4B1B68FC336A
:1028F000DC691D6AFFF7E4FF6419844204D2094BC6
:1029000001241B68002B07D004220024064B1A70F8
:10291000064A93690133936101F0A6FB200070BD64
:102920009064FF1F9809FF1F2309FF1FFC0FFF1F63
:1029300070B50C4D2B68FC335C6A01F07DFAFFF733
:10294000BFFF2B680025FC339B6AE318834204D247
:10295000054B1B68AB4200D1051B01F085FB28002D
:1029600070BDC0469064FF1F9809FF1FD722044B1B
:1029700092009B5810B5002B00D0984710BDC04660
:102980000000FF1F10B501F0DBF8FFF7EFFF27494C
:10299000274BCA6D274C1A4084235B001343CB6539
:1029A000254B1B68186A01F0DFFA244B244A1A6091
:1029B000244B254A1A60A022244B52001A60244B53
:1029C000187801F019F92000224901F02DFA0023AE
:1029D000A3600233A360204B2049236003232048D7
:1029E000A36001F021FA10221E4BFF201A60802202
:1029F00052031A60802292031A60802212041A6025
:102A000001F05AF9012001F087F9FA20400001F0A5
:102A1000B3FA582001F0D8F9134801F0DDF801208D
:102A200001F072F9072001F027FB10BD00F0004013
:102A300000FEFEFF141000409064FF1F00000340E2
:102A40000180063DBC00034034080000A4000340A0
:102A50004A0AFF1F71020000C3090000FFFF3F0088
:102A60002810004000E100E030750000674E336838
:102A700088331B6883F3088801F0CEF8644A6549FF
:102A8000136800200B401360634B644A1B68934239
:102A900000D1A6E001F0A0F90221614A13688B433E
:102AA0001360FFF76FFF5F4B5F4C1878C0B201F007
:102AB000EBF90023A3600233A3605C4B0120236089
:102AC00001F052FA0323A36001F02EFA040001F092
:102AD000E3F8050001F028FA554B186001F0B4FA4C
:102AE000544B1968621A531EA14200D2130080226F
:102AF000D203934201D39B029B0A3268D16AC90771
:102B000000D471E04C491C0C09689BB24C435943FA
:102B10002402090A641803264849FC3293680A68AB
:102B200047489B1A474A0768126847499B18474A13
:102B30009A1833409208DB190A600360042B03D90A
:102B4000013233400A6003600E684149A619300023
:102B500001F05AFA3F4F3E493B68C3183B603000D2
:102B6000019301F081F83C4E306808183849306014
:102B7000884205D9019B01333B6001F075F8316053
:102B800001F00AF9354B1B78002B0DD001F084F8C9
:102B9000334B621B196812188A4232D24919091B39
:102BA000091A304801F040F92F4E337A002B0ED02D
:102BB00001F072F8621BF1681218914224D9491988
:102BC000091B091A294801F02FF900233372284BF9
:102BD00083F3088801F078F8002001F0FDF800F098
:102BE000E3FF01F0F9F85CE7DC0199000234641AB4
:102BF0005900641A09214B438033CB40A408E418E0
:102C000089E7FA218900CCE71A49DBE79064FF1FC6
:102C10001CF00040FFFFC1FF0C0AFF1FB64121035B
:102C200010000040490AFF1F14100040C3090000B3
:102C3000100AFF1F340AFF1F380AFF1F200AFF1F58
:102C4000280AFF1F1C0AFF1F240AFF1FC4090000D7
:102C5000710200006008FF1F2C0AFF1F1C09FF1FE4
:102C6000E408FF1F00100040740BFF1F3C100040E1
:102C700000000020DC050000A022054B92009B58BC
:102C800010B5002B01D0984710BD01F005F9FBE706
:102C90000000FF1FA122054B92009B5810B5002B8E
:102CA00001D0984710BD01F0F7F8FBE70000FF1FC7
:102CB000A222054B92009B5810B5002B01D09847DB
:102CC00010BD01F0E9F8FBE70000FF1FA322054B50
:102CD00092009B5810B5002B01D0984710BD01F011
:102CE000DBF8FBE70000FF1FA422054B92009B5876
:102CF00010B5002B01D0984710BD01F0CDF8FBE7CF
:102D00000000FF1F70B500F0C7FF4F4B186001F0C7
:102D10004BF90400C30702D401F016F870BD00227D
:102D20004A4B1A604A4B18780138042829D800F019
:102D30001FFF0320181C2400200001F0C5F8012803
:102D4000ECD0444C2378042B6ED100F0C5FF002852
:102D5000E4D001F069F9582001F036F8022323701D
:102D6000DCE7200000F088FFE9E7200000F074FFB6
:102D7000E5E7200001F008F8E1E7200001F034F871
:102D8000DDE701F0D9F80500012808D1324B1B78A6
:102D9000053B012B03D82000FFF76EFFD1E72D4B39
:102DA0001B78022B01D0052B20D1022D28D12B4BD3
:102DB0009B7BAB431CD12000FFF76CFF264B1878A0
:102DC0000128BED16405BCD4244925224B7B034293
:102DD00005D1233A13405A42534126331A000B7D42
:102DE0009342AED9322001F047F8AAE7022D07D16D
:102DF000194B1B78052B11D12000FFF759FFDDE798
:102E0000012D0BD1012B03D12000FFF75FFF98E7C5
:102E1000062B03D12000FFF767FF92E7200001F0A7
:102E20003BF8022D8DD1C9E7032B04D10C4B987CC4
:102E300001F00AF872E7072B00D06FE7094B987B87
:102E400000F072FF6AE7C0469C09FF1F9809FF1F48
:102E50009009FF1F2309FF1F1C09FF1FA60BFF1F5F
:102E6000BC0BFF1FD40BFF1FFA210A4B0A4A490073
:102E70001A640A4A5A500A4A04395A50094A08310F
:102E80009A64094A5A50094A5C315A50084ADA662B
:102E90007047C0460000FF1F3528FF1F3129FF1F64
:102EA000E528FF1F1524FF1FA527FF1FB51EFF1FC5
:102EB000891EFF1FF7B50B0CFF270122009300238B
:102EC0003C001E001D009446019089B262469A4063
:102ED0001000084018413618B6B2FF2F02D1012E5B
:102EE00000D19FB2009802401A41AD18ADB2FF2C3C
:102EF00002D1012D00D19CB20133102BE6D1032069
:102F0000012E07D1012D04D1019B2401E4191C706D
:102F10000138FEBD102EFCD10238102DF9D0023040
:102F2000F7E700008023F7B59C46264B264F019318
:102F30002649274A274D284C284B02281AD160469B
:102F400038600868264E30408026360330430860DB
:102F500001990978002909D11660224A2A60224A7B
:102F60002260E02219689143A03A1BE08021C90247
:102F70001160F2E766463E600F68194E3E408027BA
:102F8000FF023E430E600199097800290DD11760B8
:102F900001280ED1154A2A60154A2260E0221968DC
:102FA0009143C03A0A431A60F7BD8021890211603B
:102FB000EEE7E0210F4A02432A600F4A22601A68B6
:102FC0008A43F0E74B0AFF1FE0000340D8000340AC
:102FD00090000340000003405000034040000340C5
:102FE000FFFFE3FF0280063D804508220180063D89
:102FF000806608220080069880550822F8B51E4B8E
:1030000080261A68002014003440324232D11A68F7
:103010001A4F32431A6001223B68063093433B60EB
:1030200000F0A2FF0122164D2B681E432E603B6864
:103030000A2613433B608027BF00124B1B683B42AC
:1030400011D1013EF6B2FF2E09D17E220E4B1C6833
:103050002B68E40B1440934323432B6005E00820C6
:1030600000F082FFE9E7002EEFD180222B68600894
:1030700093432B60F8BDC046C4F000405CF00040B4
:1030800018F0004068F0004060F0004010B501F01A
:1030900003F801215820034A00F0D6FDFFF7AEFFE8
:1030A00010BDC046600AFF1F10B5782200210348FA
:1030B00000F06AFF00F0F8FE002010BD8467FF1FDB
:1030C00070B5040000F0B8FE00230C200B4A01008C
:1030D00059438D18515C00290DD0A14208D101231C
:1030E00000246B7000F0A0FD00F0BEFF200070BD5A
:1030F00001330A2BEBD11224F6E7C0468467FF1F89
:1031000070B5040000F098FE002319001D000D4A60
:103110001078002806D0A0420CD1557001310C3235
:103120000A29F5D1002B0AD100F0BEFE00F09CFF69
:10313000002070BD5078461EB0411B18EEE700F02D
:1031400073FDF3E78467FF1FF7B504000C2000232D
:1031500084460E4D019267465F43E85D7E19A042AA
:1031600012D000280BD10A4B9C4662461B780833CC
:103170001370019B70707C557160B360FEBD0133AC
:103180000A2BE8D10320F9E70720F7E78467FF1F40
:103190008067FF1F8020F8B5484BC0051B68C1241D
:1031A0008360474BFF251A68012313434361454B56
:1031B000A4001A68444B40211A60444B1A68444BDF
:1031C0001A60444B1A59AA431A51C52292009E58BC
:1031D000AE433143802699509F583F49F6010F4036
:1031E0003E439E509E5880273602360A3043985000
:1031F00080201A5900020A4002431A5104341A5915
:10320000364E3F04324080263A431A511A59360648
:103210001202120A32431A5108341A5980260A40FF
:1032200002431A51C32292009F58B446AF4337431A
:103230009F509F58294E0F4007439F509F5837403B
:1032400080263604374380269F509F5836063F021B
:103250003F0A37439F50C0221F59AF433A431A5188
:103260001A591202120A1643C6221E5192009C5885
:10327000AC4365462C439C509C5800250C40204391
:103280009850C72080001A58154C1140C0221202D5
:103290000A431A50134B1B78DB08AB4201DC0020B9
:1032A000F8BD2378002B06D0A368002B00D09847E8
:1032B00001350C34EEE71220F2E7C0469843FF1FB9
:1032C0009443FF1FB0F000407C67FF1FB4F0004044
:1032D0007867FF1F00E100E0FF00FFFFFFFF00FF36
:1032E0008467FF1F8067FF1F030010B51F2809D8E0
:1032F000072200201340072404490A78A2431343FD
:103300000B7010BD00230620F5E7C0468067FF1F45
:10331000034A0449136800200B4013607047C046FD
:103320001CF00040FFFFC1FF054B06491B780A68EF
:1033300005485B0702401B0B134300200B607047DE
:103340008067FF1F1CF00040FFFFC1FF70B50C2518
:10335000FFF7EAFF0A4B1C780A4BE4086543ED18B7
:10336000002C01D1200070BD2B78002B06D06B689B
:10337000002B00D09847013C0C3DF1E71220F2E70A
:103380008067FF1F7867FF1F1FB5002102220B0017
:1033900001910091052000F077FE02230B490A6895
:1033A0001A42FCD120230393039B5A1E0392002B45
:1033B000FAD1074A1368002BFCDA0B246C44200076
:1033C000012100F029FE207804B010BD90C8004013
:1033D00000C8004013B504000A4B0193019B002B69
:1033E00001D1112016BDFFF7CFFF23000340044297
:1033F00005D0052000F0B8FD019B013BEDE718006A
:10340000F0E7C046FFFFFF0707B500F015FD80227B
:103410000821D205936A0191002B01D107399162ED
:1034200002210C4A11600199481E01900029FAD12D
:1034300003311160053101910199481E0190002965
:10344000FAD11160002B02D18022D205936200F0E4
:103450000BFE07BD00C00040F0B52D4C89B02378AD
:10346000002B4FD1FEF7A8FA02232A4F03903A68A7
:103470001A42FCD120230693069B5A1E0692002B6B
:10348000FAD1254E3368002BFCDA0120FFF7A2FFAA
:10349000011E02D0112009B0F0BD030003220190EB
:1034A000009005AD9F2000F0EFFD0321280000F003
:1034B000B3FD02233A681A42FCD120230793079BED
:1034C0005A1E0792002BFAD13368002BFCDA012038
:1034D000FFF780FF0028DDD10398FEF781FAAA7874
:1034E0006B7811041B020B4329780B4363601300B4
:1034F000113B0A49052B07D801239340A3600B60B9
:10350000012323700020C6E780231B03F6E7C04693
:103510008043FF1F90C8004000C800409808FF1F6C
:103520001E4B30B55A6818781D4B85B0D3185942D8
:103530004B4101210093002300F00EFC194B1A4A65
:1035400002259A6300221A6510325A658022C4212E
:103550009D65164B1648D202DA6789004258154B12
:1035600080241A4080231B041343435064234120CA
:103570000393E40500F006FA402000F003FA6562C8
:10358000039D6B1E0393002DFAD103236362FFF7A3
:103590003BFFA562FFF760FF05B030BD8C43FF1F06
:1035A00095FFFEF700C80040050001FF04E100E0C0
:1035B00000E100E0FFFF00FFF0B585B00700FEF777
:1035C000FBF9022305002D4C22681A42FCD120236E
:1035D0000093009B5A1E0092002BFAD1284E3368AC
:1035E000002BFCDA0120FFF7F5FE002803D01124A0
:1035F000200005B0F0BD234B2360022322681A424D
:10360000FCD120230193019B5A1E0192002BFAD179
:103610003368002BFCDA0120FFF7DCFE0028E6D13E
:10362000194B1F60022322681A42FCD12023029307
:10363000029B5A1E0292002BFAD13368002BFCDA4F
:103640000120FFF7C7FE0028D1D1104B23600223D1
:1036500022681A42FCD120230393039B5A1E039233
:10366000002BFAD13368002BFCDA0120FFF7B2FE01
:10367000041EBCD12800FEF7B3F9B9E790C800409A
:1036800000C8004001000006A8C8004001800001F9
:1036900010B50020FFF790FF10BD000010B5064BDD
:1036A00018705960FFF73CFF00211320034AFFF711
:1036B0004BFD002010BDC0468C43FF1F2135FF1F6E
:1036C000F0B5040085B003920291FEF775F98822E7
:1036D00063035B0B52051A438023DB059D6A80233D
:1036E000274F0092BA68002601901B039A420CD91A
:1036F000F82326001B041E401C4206D08022214BCA
:1037000052025E6219680A431A60002D0BD100F064
:1037100093FB02221C4B1A608023DB055A62013A9C
:103720009A6200F0A1FC0023039A934220D1002D5D
:103730000AD100F081FB144B03221D608023DB05BE
:103740005A629D6200F090FC8023BA681B039A4283
:1037500008D9002E06D000220A4B0C495A621A687A
:103760000A401A600198FEF73BF9002005B0F0BD51
:10377000009A0299D2181278CA540133D4E7C0468D
:103780008043FF1F00C8004000C00040FFFFFEFF55
:10379000F0B587B0029103920400FEF70DF9019095
:1037A00000F04AFB802302250122234EDB05356011
:1037B0005D629A6200F058FC204F3B682B42FCD1BE
:1037C00020230493049B5A1E0492002BFAD11C4D13
:1037D0002B68002BFCDA0120FFF7FCFD002802D04B
:1037E000112007B0F0BD2000039A029900F0BCFA46
:1037F000022304003A681A42FCD120230593059B5A
:103800005A1E0592002BFAD12B68002BFCDA0120FE
:10381000FFF7E0FD051EE3D100F00EFB802303223D
:10382000DB0535605A629D6200F01EFC0198FEF7D0
:10383000D7F8E0B2D5E7C04600C0004090C80040CD
:1038400000C80040F0B5802489B00600FEF7B4F847
:10385000E405A36A02250393029000F0EDFA012328
:10386000304F3D606562A36200F0FEFB2E4C236882
:103870002B42FCD120230593059B5A1E0592002B59
:10388000FAD12A4D2B68002BFCDA0120FFF7A2FDAC
:10389000002803D01124200009B0F0BD244B236080
:1038A000022322681A42FCD120230693069B5A1E4B
:1038B0000692002BFAD12B68002BFCDA0120FFF7CF
:1038C00089FD021EE6D11B4B03211E6003000190FF
:1038D0000090202000F0D8FB022322681A42FCD17D
:1038E00020230793079B5A1E0792002BFAD12B68BF
:1038F000002BFCDA0320FFF76DFD041ECAD100F097
:103900009BFA80230322DB053C605A629C6200F034
:10391000ABFB039B002B01D1FFF776FD0298FEF76E
:103920005FF8B8E700C0004090C8004000C8004001
:103930000100000694C8004007B50002019104226E
:10394000000A01A9FFF724FF0EBD000073B50500B2
:1039500005240B4AA3005B429B1819686B46DE1DC9
:103960003000FFF7A7FA022804D133782B55013C29
:10397000EFD276BD052CFCD00128FAD10230F8E751
:10398000140900111F2807D8012380228340D20583
:1039900091680B43936070473F2808D80123802229
:1039A00020388340D20551690B435361F3E75F2808
:1039B000F1D80123802240388340D205116A0B439D
:1039C0001362E8E71F2807D8012280218240C90539
:1039D0008B6893438B6070473F2808D80122802171
:1039E00020388240C9054B6993434B61F3E75F2858
:1039F000F1D80122802140388240C9050B6A9343E7
:103A00000B62E8E71F2810D880230200DB05153A77
:103A10001968012A06D820229143196019680A43BF
:103A20001A60704701228240F6E73F2811D88023B0
:103A30000200DB05353AD968032A06D810229143E3
:103A4000D960D9680A43DA60EBE701222038824066
:103A5000F5E75F28E5D842238022181A413B8340CE
:103A6000D205516A99435162516A0B435362D8E7B8
:103A700010B50400012813D1A022184992050B6843
:103A80005B015B0913430B60154B164A1968114023
:103A9000154A0A431A60402219680A431A6010BD89
:103AA0000028FCD101000A2000F09EFA21000B2022
:103AB00000F09AFAC0220A4B920019680A4340218A
:103AC0001A601A688A431A60B022044912060B6809
:103AD0005B015B0913430B60E1E7C04614F0004053
:103AE0001CF000407F00FEFF80FD010072B6074A17
:103AF0001368013313600422054B1A600023054A42
:103B000013608022D2055360FEE7C0467808FF1F8D
:103B1000C0F00040C4F0004005490B68002B05D1FF
:103B2000044A0A6004490A60044A13607047C046A8
:103B3000140AFF1F841E0000380AFF1FC4F0004053
:103B40000023034A1360034A1360034A136070475B
:103B500054F0004040F1004044F1004002B471468E
:103B600049084900095649008E4402BC7047C046C6
:103B700002B4714649084900095C49008E4402BC00
:103B80007047C04603B47146490840004900095ACD
:103B900049008E4403BC704701B40248844601BC0E
:103BA000604700BF5976010001B40248844601BC59
:103BB000604700BF8552010001B40248844601BC41
:103BC000604700BFE94C010001B40248844601BCD3
:103BD000604700BF19FA000001B40248844601BCE6
:103BE000604700BF8D11010001B40248844601BC4A
:103BF000604700BFDD3F000001B40248844601BCBD
:103C0000604700BFEDA5000001B40248844601BC36
:103C1000604700BFD1AE000001B40248844601BC39
:103C2000604700BFC9A9000001B40248844601BC36
:103C3000604700BF21A9000001B40248844601BCCE
:103C4000604700BF8B52010001B40248844601BCAA
:103C5000604700BF0167010001B40248844601BC0F
:103C6000604700BF0534010001B40248844601BC2E
:103C7000604700BF090E000001B40248844601BC41
:103C8000604700BF0934010001B40248844601BC0A
:103C9000604700BFA9D8000001B40248844601BCB7
:103CA000604700BFC95C010001B40248844601BC02
:103CB000604700BF6D0B010001B40248844601BC9F
:103CC000604700BFED6B010001B40248844601BCAF
:103CD000604700BF7997000001B40248844601BCE8
:103CE000604700BF01D7000001B40248844601BC10
:103CF000604700BFBD5C010001B40248844601BCBE
:103D0000604700BFC1A5000001B40248844601BC61
:103D1000604700BFE512010001B40248844601BCBF
:103D2000604700BF6911010001B40248844601BC2C
:103D3000604700BFC1F7000001B40248844601BCDF
:103D4000604700BFD9B0000001B40248844601BCFE
:103D5000604700BFDD0A010001B40248844601BC8F
:103D6000604700BFC56D010001B40248844601BC34
:103D7000604700BF9573010001B40248844601BC4E
:103D8000604700BFA1AF000001B40248844601BCF7
:103D9000604700BFF535010001B40248844601BC0C
:103DA000604700BFD544010001B40248844601BC0D
:103DB000604700BFE90B010001B40248844601BC22
:103DC000604700BFE927000001B40248844601BCF7
:103DD000604700BF7912010001B40248844601BC6B
:103DE000604700BF016C010001B40248844601BC79
:103DF000604700BFF935010001B40248844601BCA8
:103E0000604700BF8944000001B40248844601BCF9
:103E1000604700BFE9F6000001B40248844601BCD7
:103E2000604700BFC115010001B40248844601BCCF
:103E3000604700BF2D6C010001B40248844601BCFC
:103E4000604700BF75A9000001B40248844601BC68
:103E5000604700BF4DF9000001B40248844601BC30
:103E6000604700BF2144000001B40248844601BC01
:103E7000604700BF85C1000001B40248844601BC10
:103E8000604700BF6137010001B40248844601BCAD
:103E9000604700BF8914010001B40248844601BC98
:103EA000604700BFE917010001B40248844601BC25
:103EB000604700BFADAE000001B40248844601BCBB
:103EC000604700BFE9D4000001B40248844601BC49
:103ED000604700BF0134010001B40248844601BCC0
:103EE000604700BF75F8000001B40248844601BC79
:103EF000604700BFCD4C010001B40248844601BCBC
:103F0000604700BF0D52010001B40248844601BC65
:103F1000604700BFF9ED000001B40248844601BCCF
:103F2000604700BFB352010001B40248844601BC9F
:103F3000604700BF156B010001B40248844601BC14
:103F4000604700BFDD0C010001B40248844601BC9B
:103F5000604700BF116E000001B40248844601BCF6
:103F6000604700BF9D6A000001B40248844601BC5E
:103F7000604700BF0189000001B40248844601BCCB
:103F8000604700BF8512010001B40248844601BCAD
:103F9000604700BFB70E000001B40248844601BC70
:103FA000604700BF8937010001B40248844601BC64
:103FB000604700BFBD0B010001B40248844601BC4C
:103FC000604700BF8D82000001B40248844601BCF6
:103FD000604700BF2DB3001101B40248844601BC04
:103FE000604700BF51B8000001B40248844601BCDC
:103FF000604700BF859F001101B40248844601BCA0
:10400000604700BFCD0C010001B40248844601BCEA
:10401000604700BF090E000001B40248844601BC9D
:10402000604700BF3D71010001B40248844601BCF5
:10403000604700BF6DF6000001B40248844601BC31
:10404000604700BF53B9000001B40248844601BC78
:10405000604700BFC166010001B40248844601BC4C
:10406000604700BF71B0000001B40248844601BC43
:10407000604700BF9DA9000001B40248844601BC0E
:10408000604700BFF90D010001B40248844601BC3D
:10409000604700BF496D010001B40248844601BC7D
:0840A000604700BFED6801005C
:1040A80002000000CABB001101000000E0B90011C5
:1040B80002000000C6BB001101000000E840FF1F1D
:1040C80002000000E8B90011010000001462FF1F9F
:1040D80002000000C4BB0011030000008861FF1F3C
:1040E8001200000002000000CABB0011010000001D
:1040F80028BA001102000000C6BB00110100000030
:1041080025BA00110200000032BA001103000000B5
:10411800C361FF1F02000000C4BB001103000000C0
:10412800D861FF1F02000000C6BB0011010000009B
:1041380024BA00110200000030BA00110300000088
:104148009961FF1F02000000C4BB001103000000BA
:10415800BA61FF1F02000000CABB00110100000085
:1041680068BA001102000000C6BB0011010000007F
:104178003142FF1F020000007ABA0011010000005E
:1041880063BA001102000000C6BB00110100000064
:104198003042FF1F0200000078BA00110100000041
:1041A800E061FF1F02000000C6BB00110100000013
:1041B8002F42FF1F0200000076BA00110100000024
:1041C80053BA001102000000C6BB00110100000034
:1041D8002E42FF1F0200000074BA00110100000007
:1041E8004EBA001102000000C6BB00110100000019
:1041F8002D42FF1F0200000072BA001101000000EA
:1042080049BA001102000000C6BB001101000000FD
:104218002C42FF1F0200000070BA001101000000CC
:1042280044BA00110202020202020000000000006B
:104238000D0C0000354C0011F94B0011D8BA0011D3
:1042480090011D0018001800FFFF07010203040574
:104258000602010600000000000000000000000047
:104268000000000000000000000000000000000046
:104278000300000002000000CABB0011010000009A
:10428800F8BA001102000000C6BB001101000000CE
:10429800EC42FF1F0200000002BB001101000000F9
:1042A8000E62FF1F02000000C4BB001103000000E3
:1042B8007864FF1F02000000C6BB00110100000067
:1042C800EC42FF1F0200000000BB001101000000CB
:1042D8001062FF1F02000000C4BB001103000000B1
:1042E8007064FF1F120000000001000000000111AF
:1042F800FFFF000050485936000000000000000091
:104308000B000500F0000000B40000280028002879
:104318003075A000A000A000A00000080008E0017F
:10432800F0001000100010001000100010005000E5
:104338005000500010001000D007000000000000DE
:104348000F0001000500307507001000010081FF13
:1043580000000000FF0000006D710011756F001172
:10436800056D0011FFFF0100FF000000899B00118F
:10437800059900111D9800110000000000000000C0
:1043880000000800040000003B0001085902E00199
:1043980088212800FF00000002000000CABB0011AD
:1043A8000100000090BC001102000000C6BB001113
:1043B800010000001D44FF1F02000000C2BB0011E5
:1043C800010000003C68FF1F02000000C6BB00118E
:1043D800010000001C44FF1F02000000C0BB0011C8
:1043E800010000001A44FF1F02000000C6BB0011B4
:1043F800010000001844FF1F02000000BEBB0011AE
:10440800010000001044FF1F180018001D00900153
:10441800020000030202000002000000CABB0011F3
:1044280001000000A4BC001102000000C6BB00117E
:10443800010000006044FF1F02000000BCBB001127
:10444800000000000000000002000000C4BB0011D2
:0A445800030000005C68FF1F20FF56
:040000051FFF184180
:00000001FF
